:020000040800F2
:10000000101E0020010100084D5C0008D5430008C7
:100010005559000845100008298C00080000000010
:10002000000000000000000000000000656F0008F4
:10003000D32F000800000000096300087D7200084B
:100040001B010008C56000081B0100081B01000817
:100050001B0100081B0100081B0100081B01000810
:100060001B0100081B0100081B0100081B01000800
:100070001B0100081B010008F92A00081B010008E9
:100080001B0100081B010008590700081D86000815
:10009000C98600081B0100086D1000081B0100083C
:1000A0000D730008E57300081B0100081B01000820
:1000B000E9730008D17600081D7900081B010008CB
:1000C0001B0100081B0100081B0100081B010008A0
:1000D0001B0100086D8500081B0100081B010008BA
:1000E0001B0100081B0100081B010008DFF80CD0F1
:1000F00000F0F4FA0048004779A20008101E002022
:100100000648804706480047FEE7FEE7FEE7FEE7B1
:10011000FEE7FEE7FEE7FEE7FEE7FEE7997200086E
:10012000ED0000082DE9F0410024061B254671F181
:10013000000605DA01240027D0EB070067EB010178
:10014000161E73F1000605DA0027D2EB070201251F
:1001500067EB030300F0DEF986460E4617469C4621
:10016000AC4204D00025D0EB050E65EB010624B1AE
:100170000020D2EB000760EB030C704631463A4694
:100180006346BDE8F08140EA01039B0703D009E024
:1001900008C9121F08C0042AFAD203E011F8013B73
:1001A00000F8013B521EF9D2704710B5002200E062
:1001B000521C835C8C5CA34201D1002BF8D1D8B2D5
:1001C000E1B2401A10BD80EA010210B502F000430E
:1001D000400022D04A001FD0010E01EB1261C0F393
:1001E0005600C2F3560240F4000042F40002A0FBA5
:1001F000022000047F39140400D0401C50EA124051
:1002000001D44000491EC2B20C0604EBD010401CC1
:100210004008802A02D003E0002010BD20F0010039
:10022000002900DA0020184310BD2DE9FE4F81EAB5
:10023000030404F0004421F0004100944FF0000B4F
:1002400023F0004350EA01045ED052EA03045BD07D
:10025000C3F30A54C1F30A552C44A4F2F3340194B5
:10026000A0FB0254C1F3130141F48011C3F3130343
:1002700043F4801301FB024400FB034E840A970AF7
:1002800044EA815447EA8357A4FB076802958D0A24
:1002900005FB07854FEA932C04FB0C542705029DB0
:1002A0004FEA065847EA1637B5EB08056EEB070C20
:1002B000870E920E47EA811742EA8312A7FB0201DA
:1002C000B6EB0B0164EB00042B0D43EA0C335E1814
:1002D00044EB1C50DA465146E7FB0201C5F3130418
:1002E0004FEA0B3343EA14534FEA0432019C43EACA
:1002F0000603A4F10C040294009CCDE900B400F0C4
:100300009FF903B0BDE8F08F00200146F9E72DE921
:10031000F04D81EA030404F0004B21F0004514463F
:100320004FF0000A23F0004150EA050220D054EAC1
:1003300001021DD0C5F30A570246C5F31303C1F3EA
:100340001300C1F30A5640F4801543F48013A7EB61
:100350000608101BD64608F2FD3873EB050002D3E1
:1003600008F1010801E092185B41B8F1000F03DACF
:1003700000200146BDE8F08D00204FF480110646B4
:1003800084460EE0171B73EB050705D3121B63EBC6
:10039000050306434CEA010C49084FEA3000921865
:1003A0005B4150EA0107EDD152EA030012D082EA24
:1003B000040083EA0501084305D0101BAB4106D2B7
:1003C0000122002306E000224FF0004302E06FF01C
:1003D000010253101AEB06004CEB085110EB0A0017
:1003E00041EB0B01BDE8F04D00F01BB970B521F0F9
:1003F000004303430CD0C1F30A550024D5EB040598
:1004000064EB0403D617AD1AB34102DB00200146AA
:1004100070BD201841EB025170BDC10F80EAE07041
:100420000844CA079623002100F0CDB89623002285
:10043000114600F0C8B80EB5C10F80EAE07008445C
:10044000CA07002140F233438DE80E000A460B46EE
:1004500000F0F6F803B000BD0EB540F23341029152
:100460000021CDE900110A460B4600F0E9F803B07F
:1004700000BD00F0004220F00040C10DC0F31600A6
:1004800040F400007F2901DA00207047962903DC40
:10049000C1F19601C84001E096398840002AF4D0A5
:1004A0004042704770B5C1F30A5201F00045002484
:1004B000C1F3130140F2FF3341F480119A4201DA93
:1004C000002070BD40F233439A42A2F2334203DC73
:1004D000524200F05FF800E090402C43F1D04042DF
:1004E00070BDC1F30A5210B5C1F3130140F2FF33DE
:1004F00041F480119A4201DA002010BD40F23343EA
:100500009A42A2F2334203DC524200F043F810BD9B
:10051000904010BD2DE9F05F0546002092469B46B5
:1005200088460646814640241BE028464146474609
:10053000224600F02FF853465A46C01A914110D374
:1005400011461846224600F016F82D1A67EB0108EE
:100550004F4622460120002100F00DF817EB00095C
:100560004E41201EA4F10104DFDC484631462A46F4
:100570004346BDE8F09F202A04DB203A00FA02F14E
:10058000002070479140C2F1200320FA03F3194381
:1005900090407047202A04DB203A21FA02F0002123
:1005A000704721FA02F3D040C2F120029140084383
:1005B000194670470029A8BF7047401C490008BF72
:1005C00020F00100704710B4B0FA80FC00FA0CF083
:1005D00050EA010404BF10BC704749B1CCF12004BB
:1005E00021FA04F411FA0CF118BF01212143084348
:1005F000A3EB0C01CB1D4FEA00614FEA102042BF74
:10060000002010BC704700EBC35010440029A4BF69
:1006100010BC7047401C490008BF20F0010010BC0E
:10062000704710B5141E73F1000408DA401C41F144
:10063000000192185B411A4301D120F0010010BD66
:100640002DE9F04D92469B4611B1B1FA81F202E0DC
:10065000B0FA80F220329046FFF78DFF04460F4635
:1006600040EA0A0041EA0B0153465A46084313D0B8
:10067000114653EA010019D0C8F140025046FFF775
:1006800089FF05460E46504659464246FFF773FF1E
:10069000084305D0012004E020463946BDE8F08D2E
:1006A0000020054346EAE0762C4337430A98630569
:1006B000E40AA0EB08000022FD0A44EA47540A308D
:1006C00002D500200146E9E7010510196941DDE97D
:1006D000084500196941BDE8F04DA2E7064C074DF9
:1006E00006E0E06840F0010394E807009847103402
:1006F000AC42F6D3FFF7FEFCE0C6000800C70008D6
:1007000070B58C1810F8015B15F0070301D110F8D3
:10071000013B2A1106D110F8012B03E010F8016B00
:1007200001F8016B5B1EF9D12B0705D40023521E83
:100730000DD401F8013BFAE710F8013BCB1A921CEB
:1007400003E013F8015B01F8015B521EF9D5A142E9
:10075000D8D3002070BD00002DE9F0415C4C4FF46F
:1007600090652946204600F044FA00287ED02946AC
:10077000204600F0CBF857490888401C088001212A
:10078000204600F015FB544842F21072B0F85810A1
:10079000914202D2491CA0F8581009F0A9FF4F4D10
:1007A000B5F91410B5F9120008F032FC4C4CA5F85C
:1007B00056002080A16820468847A088A5F85800E8
:1007C00005F018FB0AF094F8464E474C307808289C
:1007D0002ED045F6AC30606042F6EF60A06042F289
:1007E000C400E0604148008A2080208E6080A16BB8
:1007F0003D488847208E40F21C7180003C4C00EB45
:1008000081006887207A4FF0000740073CD5394DBA
:1008100040F21A61E888401C80B2E880884250D3D8
:100820004FF48051344803F03DF8012809D048E0E6
:1008300041F2130060604FF48060A06040F61B50EE
:10084000CFE72E49EF802E480A780A2A03D2438840
:100850000BB9521C0A70D1B2022932D84188F9B9B9
:10086000A16821F00401A160264900E02DE0CA88BA
:1008700022F40062CA80017821F00201017022494D
:1008800049F6816008801CE030780A2815D2DFE83C
:1008900000F0140508180B180E14110808F08EFD4E
:1008A0000FE00AF069FA0CE00BF000F9F9E704F048
:1008B0002DFB06E009F0B6FAF3E701F081FE84F8BB
:1008C000BA70BDE8F0410AF039B8BDE8F081000027
:1008D0000024014078070020500100206000002023
:1008E000600700206F070020E000002008020020C1
:1008F000C0020020100B0020000C01408B020020E1
:1009000010060020480C0020442C01406FEA112101
:10091000016070470029816802D041F0010101E0C7
:1009200021F00101816070470029816802D041F403
:10093000807101E021F48071816070472DE9F04100
:10094000854E92B0304600F011F90BA800F03FFA46
:1009500001214FF4C06005F06BFD00248DF831409B
:100960004FF46020CDE90D044FF4A0204FF00A08A9
:100970000B9001278DF83C808DF830700BA9304624
:1009800000F086F9754D8DF831408DF830708DF896
:100990003C700BA9284600F07BF901231A460F2171
:1009A000304600F0C6F9022201231146304600F01D
:1009B000C0F9012303221946304600F0BAF9012399
:1009C00004220021304600F0B4F90123052203215E
:1009D000304600F0AEF9012306220821304600F02F
:1009E000A8F9012307220A21304600F0A2F90123C9
:1009F00008220B21304600F09CF9012309220D2129
:100A0000304600F096F901230A220421304600F016
:100A100090F90121304600F084F90121284600F0C8
:100A200080F901231A460521304600F055F90123CB
:100A30001A460621284600F04FF90021304600F002
:100A4000CBF84FF4E041284600F0C6F801213046CB
:100A500000F0B8F80121284600F0B4F80121304632
:100A600000F0A6F80121284600F0A2F80121304646
:100A700000F09EF90121284600F09AF940F6145141
:100A8000374807F022FA12208DF8400002208DF836
:100A900041008DF842408DF8437010A805F004F92C
:100AA00001224FF49061304600F0E8F80121304611
:100AB000FFF73AFF01213046FFF72CFF01212846BE
:100AC000FFF728FF304600F06EF9304600F09FF83F
:100AD0000028FAD1304600F075F9304600F082F86F
:100AE0000028FAD1284600F05EF9284600F08FF879
:100AF0000028FAD1284600F065F9284600F072F87F
:100B00000028FAD10121084605F06EFC154D284653
:100B100002F02EF8684602F0CEF80F4801A94C30DA
:100B20000090114881E811018020CDE90440400087
:100B3000069080000790202008904FF44050CDE9A7
:100B400009046946284602F099F80121284602F076
:100B500003F812B0BDE8F0810024014000280140F4
:100B6000002C014008000240D00200200D4910B5C1
:100B7000884202D1012144150AE00B49884202D182
:100B80000121041504E0094988420AD10121CC035E
:100B9000204605F059FC2046BDE81040002105F034
:100BA00053BC10BD0024014000280140003C01401E
:100BB0000029816802D041F4801101E021F4801104
:100BC000816070470029816802D041F4004101E052
:100BD00021F4004181607047826822F4E0420A43B8
:100BE00082607047014600208968490700D50120CE
:100BF000704710B50246002054680B0AC9B20C4079
:100C00001168194202D0002C00D0012010BD01460D
:100C100000208968090700D50120704738B50121F7
:100C20001C2005F005FCEF20ADF8000000248DF835
:100C3000034003258DF8025069460D4802F0B4FDCB
:100C40000120ADF800008DF803408DF80250694690
:100C5000084802F0A9FD3B20ADF800008DF80340E4
:100C60008DF802506946044802F09EFD38BD000030
:100C700000080140000C014000100140002A4268B9
:100C8000C9B201D00A4300E08A43426070470000C5
:100C900010B542680E4B0C791A400B6842EA0422E8
:100CA0001343436083680B4A1340D1E90242224355
:100CB0004C7943EA44031A438260C26A097C22F4F5
:100CC0007002491EC9B242EA0151C16210BD000062
:100CD000FFFEF0FFFDF7F1FF70B5072409290AD9DF
:100CE000C568A1F10A0606EB4606B440A543B34029
:100CF0001D43C56007E0056901EB4106B440A5430B
:100D0000B3401D430561836BC3F30154121B921C56
:100D100002EB82041F22A2409343A1400B43836352
:100D200070BD826B491E22F4401242EA0151816378
:100D3000704770B5072409290AD9C568A1F10A06C8
:100D400006EB4606B440A543B3401D43C56007E02B
:100D5000056901EB4106B440A543B3401D4305615D
:100D60001F23072A09D2446B521E02EB82029340D2
:100D70009C4391400C43446370BD0D2A09D2046B1F
:100D8000D21F02EB820293409C4391400C430463C8
:100D900070BDC46A0D3A02EB820293409C439140BD
:100DA0000C43C46270BD816841F0080181607047E6
:100DB0000029816802D041F4A00101E021F4A001E2
:100DC00081607047816841F00401816070470021B3
:100DD0000160017141718160C1600121017470473E
:100DE000002800DA4042B0F5803F02DB4FF6FF708A
:100DF000704780B27047401AB0F5004F02DBA0F593
:100E00008030704710F5004FFBDA00F580307047F6
:100E100070B51E4C214694F83800B1F842500628AF
:100E20001ED9B4F84A10B4F84C00A1EB000202F14C
:100E30000902122A04D8FFF70FFB0022144B0AE024
:100E4000884204D2FFF708FB0022124B03E0FFF7B1
:100E500003FB0022104BFFF7E8F9FFF742FB09E024
:100E600005D12846FFF7F8FA0C4A0D4BF3E70D4978
:100E700051F82000C5EB45116063B0EB410F03D979
:100E8000C5EB45104000606370BD00007404002095
:100E9000000034400000334000003540676666665D
:100EA00066E64B4058BD000810B50C4C2078400752
:100EB00013D5FFF7ADFF0A49A08E088008483038E7
:100EC000018821F010010180001F018841F010010C
:100ED0000180207820F00400207010BD74040020F0
:100EE00040040040F0B4294A294C0021137A02F151
:100EF000380033B1B4F9023041F2CD05AB421EDC0B
:100F00001172224E8368234D3836C3F3C00CC3F3ED
:100F1000002736686D6CBC4519D1360711D5267887
:100F200026F002062670012651831672A180C16246
:100F3000642D06DAD90506D443F0080105E0A18046
:100F4000C162F0BC704723F00801816018E090F89E
:100F50004A40C4B9B5F5966F15DC340713D4548BE9
:100F6000B4F5FA6F02D2641C5483EAE70A4A67F3C5
:100F7000C303147824F0010414705180118283603B
:100F8000F0BC08F03BBD5183DBE700008802002085
:100F90001006002050010020F80A0020012180F8EE
:100FA0002E104FF4AF6101861F21418645F2715129
:100FB0008186704770B506464089204B204C4FF41F
:100FC0000051002580B362887AB1012A0CD1E188F2
:100FD000491C89B2E1803289914205D36580E58060
:100FE000FF2801D0401E708170BD70882288904219
:100FF00001D9012200E00022184602F05EFC708850
:10100000B18801442088401C80B220808142EBD806
:101010002580A088401C80B2A080F1888842E3D35C
:1010200001206080A58070BDFFE70022184602F015
:1010300044FCA580E58025806580F4E70010014030
:10104000F0050020FEE7000010B5074C0021204607
:1010500000F06AF80121204600F066F82046BDE85D
:101060001040022100F060B80064004010B50D4C43
:101070000B49204600F06AF809492046891C00F017
:1010800065F80949204600F061F8084C206808F02E
:10109000B5F9002106A009F029FA206010BD000072
:1010A0000200F010006400407000F0307C08002066
:1010B0006465765F63616E310000000070B51848AA
:1010C000017861F30704417861F30F24817861F3BB
:1010D0001744C17861F31F640179407961F3070512
:1010E00060F30F2502F04AF90E4E304602F0C4F8C4
:1010F000A1B2304602F0FCF8210CB01C02F0F8F866
:10110000A9B2301D02F0F4F805482838C07800F084
:101110000301B01D02F0ECF8BDE8704002F0E0B849
:10112000D707002000A0030841B101290AD00229F5
:1011300003D1816841F4000181607047816841F00A
:101140008001F9E7816841F40041F5E70A4A9142DC
:1011500002D1002181617047C1F313028B0101D5D7
:10116000C26070474B0101D502617047090101D58A
:1011700082607047426070477000F03030B50823DD
:1011800010240422B1F5007F1DD010DC202929D0C5
:1011900007DC012921D0042922D0082900D1C4600C
:1011A00030BD402920D0B1F5807FF9D10BE000257A
:1011B000B1F5004F06D008DCB1F5806F03D0B1F572
:1011C000006FEDD18561426030BDB1F5803F0DD03B
:1011D000B1F5003FF8D1446030BD0549816030BDB4
:1011E000C36030BD036130BD046130BD436030BDBC
:1011F000010101003EB5684600F026FA00208DF896
:10120000080001218DF809108DF80A008DF80B10E7
:101210008DF806001D498DF807008DF8020001F1D8
:101220001000897C8DF80310C1788DF804100179C5
:101230008DF80510C088164CADF8000069462046B0
:1012400000F045F901220221204600F038F9012280
:101250001146204600F033F90E492046FFF776FF8D
:101260000C492046891CFFF771FF0B492046FFF708
:101270006DFF08492046491EFFF768FF01224FF421
:101280000441204600F01BF900203EBD8C080020E0
:10129000006400400200F0107000F030094910B501
:1012A00088424FF0010101D14C0601E04FF080640B
:1012B000204605F0B1F82046BDE81040002105F0B9
:1012C000ABB80000006400402DE9FF470026012173
:1012D00019488DF80B608DF80C10DFF86090ADF8B0
:1012E00008608DF80D10354634464FF0040809F1BA
:1012F000800AC7681AE000BF8DF80A4059F8261026
:10130000761C480BADF8000008EBC101ADF80210E7
:101310005AF825106D1C4A0BADF8042008EBC100EB
:10132000ADF80600684600F00BF8641CBC42E3DB35
:1013300004B00020BDE8F08778080020FC180020E9
:10134000F0B5827A012191402E4A136843F00103DF
:1013500013602C4B1C331C688C431C60294D067B8E
:10136000294C0C35A6B92E688E432E604688C78856
:1013700046EA0746877A04EBC707C7F8406606883F
:10138000878846EA0746877A04EBC707C7F84466AA
:10139000067B012E12D12E680E432E60867A0568D8
:1013A00004EBC6064FEA3545C6F84056867A4568CE
:1013B00004EBC6044FEA3545C4F84456114CC57ACF
:1013C000241D002D256806D00D4325600D4C058990
:1013D000143415B104E08D43F7E725688D4325608B
:1013E0000589012D02D125680D432560407B012828
:1013F00002D1186808431860106820F001001060DE
:10140000F0BD000000660040006000400246002081
:1014100053690B424AD0B1F5807F3BD013DC0829D9
:101420002ED007DC012926D0022927D004293DD15E
:10143000D0682BE0102925D0202926D0402935D18D
:101440001069102130E0B1F5004F2BD00BDCB1F565
:10145000007F22D0B1F5806F22D0B1F5006F25D189
:101460009069702120E0B1F5803F11D0B1F5003FC7
:101470001CD15068E5E790680D4915E0D06802E09E
:10148000D068DEE7106903210EE0106908210BE047
:101490005068FBE79069012106E09069022103E0B2
:1014A000906900E05068042101F064B870470000C2
:1014B000010101008069C0F3021000017047002A99
:1014C000426901D00A4300E08A434261704710B587
:1014D0000368002223F002030360036843F0010362
:1014E00003604FF6FF7300E0521C4468E40701D12B
:1014F0009A42F9D14268D2073ED08A79012A02681D
:101500003CD022F080020260CA79012A026838D0F9
:1015100022F0400202600A7A012A026834D022F0E6
:10152000200202604A7A012A026830D022F01002BA
:1015300002608A7A012A02682CD022F00802026036
:10154000CA7A012A026828D022F0040202608A784E
:10155000CC78920742EA04620C7942EA04424C7960
:10156000098842EA0452491E0A43C261016821F017
:1015700001010160002114E0002010BD42F0800252
:10158000C1E742F04002C5E742F02002C9E742F05D
:101590001002CDE742F00802D1E742F00402D5E79D
:1015A000491C4268D20701D09942F9D14068C0076E
:1015B000E2D1012010BD000010B500EB0113D3F8FB
:1015C000B04114F004041472D3F8B04134D0E408EC
:1015D000C2F80440D3F8B04104F002045472D3F8C6
:1015E000B44104F00F049472D3F8B441240AD474C3
:1015F000D3F8B841D472D3F8B841240A1473D3F89D
:10160000B841240C5473D3F8B841240E9473D3F822
:10161000BC41D473D3F8BC41240A1474D3F8BC4140
:10162000240C5474D3F8BC311B0E937439B1016986
:1016300041F02001016110BD640D1460CAE7C1686A
:1016400041F02001C16010BD00218171C1710172A2
:1016500041728172C1728170C170032101710221D6
:10166000417101210180704730B502460020936826
:101670005B0108D49068000101D5012003E0906867
:10168000C00037D5022002EB0012D2F8803103F0FF
:101690000103C2F880310B7A73B3D2F880414D68F0
:1016A0001C434B7A43EAC5031C43C2F880418B7A42
:1016B00003F00F038B72D2F8843123F00F03C2F8CA
:1016C0008431D2F884318C7A2343C2F88431CB7AC6
:1016D000CC6843EA0423C2F88831CB7B096943EA2A
:1016E0000121C2F88C11D2F8801141F00101C2F839
:1016F000801130BD042030BDD2F880314C7A2343B4
:101700000C8843EA4453C2F88031D0E72DE9F04F0A
:10171000FE4885B0416C1A20B1FBF0F086B20D2076
:10172000B6FBF0F8FA48FB49B0F91A00C0F30F1005
:101730000490B1F91020C82042434FF47A7000EBB6
:10174000A2339CB2092303EBA232132A00D204462F
:101750008B460D46B1F91E0001F080F90390B5F9F2
:10176000200001F07BF90290B5F9220001F076F932
:10177000E94B0190D88B4FF4FA71484340F6FF7162
:10178000B0FBF1F0DFF894C31FFA80F9E44DBCF828
:101790001000E4490090E8880A78070967F300021E
:1017A000C70A67F34102C70867F38202870867F335
:1017B000C302070B67F30412470867F3451260F38F
:1017C0008612470B67F3C7120A704A78470A67F315
:1017D0000002470967F34102870967F38202070A9B
:1017E00067F3C302C70967F30412AF7ABF0867F350
:1017F0004512800B60F386124A7093F8070110B10E
:1018000042F0800001E022F080004870C4489A460F
:10181000027B887862F341001A89D50885EA12258F
:10182000ED4365F382009CF8005065F30410550900
:1018300065F34510D20A62F38610887093F84A2047
:101840002AB1012A07D0022A0AD0032A0DD0CA7869
:1018500022F003020CE0CA7822F00302521C07E0D7
:10186000CA7822F00302921C02E0CA7842F0030216
:10187000AC4BCA702833A3F118059A7802F0030222
:10188000012AAA7812D022F01002AA70CA7897070B
:101890000FD020F008008870A2482830407900F06E
:1018A0000300012808D0022809D00BE042F0100202
:1018B000EBE740F00800EEE742F0040001E022F020
:1018C0000400C87098480278964F791DF87862F342
:1018D000041020F08000F8703246381D05F0CAFC74
:1018E000924EB6F9020006F09BFBB871B6F90400FF
:1018F00006F096FBF87107F10806711C3046049A51
:1019000005F0B8FC2246F11CB01C05F0B3FC884879
:101910006421B0F904004843800B03F047FC707168
:101920004A46F11DB01D05F0A5FCBBF91000FFF7FC
:1019300057FAC8214843000C03F038FC287006F120
:101940002000012401780227B4EB911F03D1A9786C
:1019500041F0010105E0B7EB911F03D1A97821F017
:101960000101A970437803F00301012902D0022983
:1019700004D007E0A97841F0020102E0A97821F043
:101980000201A970DAF80810AA784FEAD11C6CF3AA
:101990008202AA7090F802C05646CCF3810CBCF1CA
:1019A000010F03D0BCF1020F03D005E042F020028A
:1019B00001E022F02002AA708346A246B4EB931FF6
:1019C00003D1D0B240F0800004E0B7EB931F02D106
:1019D00002F07F00A8705748DFF84491514C427FD5
:1019E000E878183462F34100CA0A62F3820096F87C
:1019F0002A2162F30000327962F3C300E87099F89B
:101A00000C3028794A4663F3820033785B115B1C03
:101A100063F3C3004B0963F3041028710816697956
:101A2000401C60F3C301697199F80010E87961F313
:101A30000300D1884246C90B61F3861099F80A1059
:101A4000C90861F3C710E871611C204605F012FC5B
:101A5000E11CA01C009A05F00DFCB6F9E800FFF7A8
:101A6000BFF9C8214843800B03F0A0FB2071307AF6
:101A7000C109A07961F3C710B6F8C8100A0A62F369
:101A80000600A071E171273C611C2046039A05F015
:101A9000F1FBE11CA01C029A05F0ECFB611D201D6E
:101AA000019A05F0E7FB84F806809BF800005C468D
:101AB00020F00C00001D20F03000103020F0C0019C
:101AC00040318BF800109BF8010020F00300401C0F
:101AD00020F00C00001D20F0C00340338BF80130D3
:101AE000A078DFF840B020F00300401C20F00C008C
:101AF000001DA0708646E078ABF11F0B20F0E002DD
:101B00004032E2709BF80000002815E050010020F0
:101B1000EC04002058050020C0020020F80A002034
:101B2000480C0020AF07002008060020440E0020CB
:101B3000100600206C0E00207ED0F07B00287BD1A8
:101B40008BF800000BF1170090F800C00CF0030CAC
:101B5000BCF1010F06D090F800C00CF0030CBCF1F2
:101B6000020F04D190F800C06CF3010121700178DC
:101B7000C1F38101012904D00178C1F38101022957
:101B800006D101784FEA910C21786CF38301217022
:101B90000178C1F30111012904D00178C1F30111C9
:101BA000022906D101784FEA111C21786CF3051146
:101BB000217090F800C05146BAEB9C1F04D090F8F9
:101BC00000C0B7EB9C1F09D190F800C04FEA1C1869
:101BD00094F800C068F3871C84F800C090F801C036
:101BE0000CF0030CBCF1010F06D090F801C00CF012
:101BF000030CBCF1020F04D190F801C06CF3010397
:101C000063704378C3F38103012B04D04378C3F39B
:101C10008103022B06D143784FEA930C63786CF36F
:101C2000830363704378C3F30113012B06D0437819
:101C3000C3F30113022B00E028E106D143784FEAF9
:101C4000131C63786CF3051363704378B1EB931F37
:101C500003D04378B7EB931F06D143784FEA131CA8
:101C600063786CF387136370837803F00303012BAD
:101C700004D0837803F00303022B05D190F802C04F
:101C800073466CF30103A3708378C3F38103012BC4
:101C900004D08378C3F38103022B06D183784FEA03
:101CA000930CA3786CF38303A3708378C3F30113BD
:101CB000012B04D08378C3F30113022B06D1837860
:101CC0004FEA131CA3786CF30413A3708378B1EB71
:101CD000931F03D08378B7EB931F06D18378C3F3A8
:101CE000011CA3786CF34713A370C378DB0608D0FC
:101CF000C37803F01F031F2B03D2C37863F30402DE
:101D0000E270C278520905D0C2785309E27863F3D1
:101D10004712E270027902F00302012A04D002792C
:101D200002F00302022A04D10279237962F301034B
:101D300023710279C2F38102012A04D00279C2F32D
:101D40008102022A05D102799308227963F3830282
:101D500022710279C2F30112012A04D00279C2F37E
:101D60000112022A05D102791309227963F30512BF
:101D700022710279B1EB921F03D00279B7EB921F67
:101D800005D102791309227963F38712227142790E
:101D900002F00302012A04D0427902F00302022A6F
:101DA00004D14279637962F3010363714279C2F32A
:101DB0008102012A04D04279C2F38102022A05D1AC
:101DC00042799308627963F3830262714279C2F3C4
:101DD0000112012A04D04279C2F30112022A05D16C
:101DE00042791309627963F3051262714279B1EBAA
:101DF000921F03D04279B7EB921F05D142791309A4
:101E0000627963F387126271827902F00302012A18
:101E100004D0827902F00302022A04D18279A379E4
:101E200062F30103A3718279C2F38102012A04D013
:101E30008279C2F38102022A05D182799308A279BC
:101E400063F38302A2718279C2F30112012A04D0E2
:101E50008279C2F30112022A05D182791309A2798B
:101E600063F30512A2718279BAEB921F03D08179D4
:101E7000B7EB911F05D181790A09A17962F3871126
:101E8000A171C179E07961F30300E071DFF840816D
:101E900098F8000000F00F00042801D1FFF70EF9B8
:101EA0002078C0F38100012832D0A87820F0040007
:101EB000A870484AA978107F8B074FF47F4142D51C
:101EC000802821D3444B00F01F00126853F82000F3
:101ED000024219D1B06840F08070B0603C483038A0
:101EE0008078C00733D0B068C00130D53B48406C23
:101EF00032282CD85F46BBF802008B46584547D1A4
:101F000001F0F8FC788024E0B06820F08070E4E70D
:101F100098F8070001060CD500F07F00142808D8B7
:101F2000A87840F00400A870A87920F00300801C75
:101F300007E0A87820F00400A870A87920F003003A
:101F4000401CA871B5E7B06820F08070B060ABF8B5
:101F50000210A878800703D4B06820F08070B060C9
:101F6000607810F0300F02D00020A9F80C0098F82B
:101F70000400C00701D0A9F80CA099F80C00C10713
:101F80001348A0F14900017812D041F0010111E09D
:101F900001F098FC40F6B8318842DAD3B068C1014C
:101FA000D7D50005D5D4A9F80CA0A7F802B0D0E782
:101FB00021F001010170B168C901017802D541F039
:101FC000020101E021F00201017005B0BDE8F08FCF
:101FD000DF07002018060020B8C1000850010020CB
:101FE00070B51548006810F0E05F23D0134CD4E9B9
:101FF000001081421ED004EB001104F5A1608A6834
:1020000042600A7B827204230372002545720B3002
:102010000E31FEF7B8F872B66068401C6060402868
:1020200000D3656062B60649BDE8704002480838D2
:10203000FFF71ABB70BD000008640040F4140020D4
:10204000FC19002030B5002300280CDA002904DD3B
:10205000404202B24FF4804303E04942224B09B2AE
:1020600002460846114643F233324FF40074002909
:1020700008DD904201DD91420ADCA04214DAA1425F
:102080000EDB11E0904206DD43F23332D14202DA38
:102090004010491008E0A04206DA11F5007F03DD88
:1020A0000001090100B209B2104D0022002941FAD5
:1020B00002F408DD04441041081A01B235F8120098
:1020C00024B2184407E0041B1041084401B235F85B
:1020D000120024B2181A521C03B2D2B220460B2AA4
:1020E000E4D398B230BD000000C0FFFF4CBC000834
:1020F000FCB505464FF6FF7600200C46ADF80060B3
:1021000048F205078DF8040020E000BF15F8010B28
:102110008DF8040001A9084602F0D4FDBDF80000C6
:102120009DF8041080EA0120ADF800005FF0000087
:10213000BDF800100A0402D587EA410101E006EA71
:102140004101401CADF800100828F1DB641EDDD20F
:102150006946084602F0A0FDBDF80000FCBD000085
:102160000246002004E000BF12F8013B1844C0B250
:10217000491EF9D27047000070B5144A85B0108826
:102180000024134901940094039420460494138876
:1021900007E0CD8B009E354400950D8B019E3544A4
:1021A000019515889D42F4D0401CC0B28028EED322
:1021B00000984111074841808480019841110648E8
:1021C00081830183818205B070BD00007807002003
:1021D000C002002010060020EC04002030B4104C97
:1021E000002003464FF47F42A4F1340121F810305F
:1021F00024F81020401C1A28F8DB0A4B002000BFEE
:1022000033F8104021F81040401C1A28F8DB06482B
:1022100006490280012081F8300030BC03F09CBBED
:10222000B8100020380800206C080020180F00208B
:102230002DE9F84303F0E2FBC64DC54B00204FF4F7
:102240007F4105F1340400BF35F8106033F81020E9
:10225000964203D025F8102024F81010401C1A28AC
:10226000F2DBBD4890F83000012808D05FF0000094
:1022700024F81010401C1A28FADBBDE8F88303F09C
:102280003DF8208801F01EFB2988B44E88420AD30D
:1022900001F030FB2080B24800906B460822B14923
:1022A000306809F0B1FC608801F00CFB6988884255
:1022B0000CD301F01FFB6080A948AA49401C009084
:1022C0006B4608220831306809F09EFCA08801F0B6
:1022D000F9FAA98888420CD301F00CFBA080A04831
:1022E000A049801C00906B4608221031306809F02C
:1022F0008BFCE08801F0E6FAE98888420CD301F013
:10230000F9FAE08096489749C01C00906B46082275
:102310001831306809F078FC208901F0D3FA298956
:1023200088420CD301F0E6FA20818D488D49001DCA
:1023300000906B4608222031306809F065FC608906
:1023400001F0C0FA698988420CD301F0D3FA6081A8
:1023500083488449401D00906B460822283130682C
:1023600009F052FCA08901F0ADFAA846A989052719
:102370007D4D884216D36878052813D201F0BAFA49
:10238000A0816878401CC0B26870052800D96F70C1
:1023900073487449303000906B4608223031306801
:1023A00009F032FCE08901F08DFAB8F80E1088428D
:1023B00016D3A878052813D201F09CFAE081A878FA
:1023C000401CC0B2A870052800D9AF7064486549A8
:1023D000313000906B4608223831306809F014FC27
:1023E000208A01F06FFAB8F81010884216D3E87806
:1023F000052813D201F07EFA2082E878401CC0B292
:10240000E870052800D9EF705548564932300090E1
:102410006B4608224031306809F0F6FB608A01F013
:1024200051FAB8F81210884216D32879052813D229
:1024300001F060FA60822879401CC0B2287105283A
:1024400000D92F7146484749333000906B46082227
:102450004831306809F0D8FB208D01F033FAB8F824
:102460002810474688420BD301F044FA20853F48A4
:102470003C4900906B460822A031306809F0C4FB4B
:10248000608D01F01FFA798D88420CD301F032FA89
:10249000608536483349401C00906B460822A831BD
:1024A000306809F0B1FBA08D01F00CFAB98D8842BB
:1024B0000CD301F01FFAA08529482A49503000901A
:1024C0006B460822B031306809F09EFBE08D01F0C8
:1024D000F9F9F98D88420CD301F00CFAE085204817
:1024E0002049603000906B460822B831306809F00E
:1024F0008BFB208E01F0E6F9398E88420CD301F077
:10250000F9F9208616481749613000906B46082279
:10251000C031306809F078FB608E01F0D3F9798E14
:1025200088420CD301F0E6F960860D480D4962300F
:1025300000906B460822C831306809F065FB0C48F2
:10254000FEF7B8FF00283FF498AE287095E600002B
:102550003808002084100020180F00207C0800207C
:102560000002FF184C0F0020700800200006FF1822
:1025700000640040024600200A4200D0012070475B
:1025800030B50E4902880A800C4A4388083A138005
:102590000B1F808818802024151F2C800020401CD1
:1025A00080B23C28FBD341F69910088044F64800DD
:1025B000108046F6480018802C8030BD202C014049
:1025C000114944F648000880091D46F64800088075
:1025D000091D41F6991008800B48001F018841F041
:1025E0002001018009480021A0F86810A0F86610B9
:1025F000A0F86410A0F86210A0F86010A0F85E10B7
:102600000348418181827047182C0140C00200209C
:10261000600000202DE9F047494B4A480021DA7A52
:102620000778802A27F0010675D31C68464B02F014
:102630001F0253F82220454B14421A6802D042F080
:10264000200201E022F0200299461A60404B3F4DE3
:10265000DFF800A11C78404B95F84A50022CB3F9E2
:1026600004305AD1D9F808C0CCF3C004CCF3002808
:10267000444552D0354C383C94F80480B8F1000FF2
:1026800006D0B8F1010F0DD0B8F1020F4AD120E009
:10269000110547D5910645D40121217127F0040188
:1026A00001703FE016053DD496063BD57E0739D430
:1026B00046888EBB4380002B09DD47F00501017081
:1026C000022121712549B1F8441001822AE02171CB
:1026D00028E0C7880FB9002B16DC077BAF4213D167
:1026E0001F4FFF895FEA47780ED45FEA87780BD4E3
:1026F0005FEA427808D55FEA826805D5FF0703D113
:1027000015B15FEACC170DD506704180AAF800100C
:1027100041810182DBE70EE004E006704180AAF807
:1027200000104181C3800573500960F3CB22C9F8C2
:102730000020BDE8F087067041804181F9E7000084
:1027400018060020F80A0020B8C10008C0020020C6
:102750006F070020200100201006002050010020FB
:10276000480C00202DE9F04F97B000240C940D94F4
:102770000E940F9472B6B148816941F40071816181
:10278000816941F4806181614FF4004003F022FED1
:10279000AB4E00213046FEF7C7F800213046FEF769
:1027A000B9F80021A748FEF7B5F8A74F0021384631
:1027B00000F0D2F901204FF47041401C8842FCD354
:1027C0003046FEF7D3F99F48FEF7D0F9B9463846B0
:1027D00000F0CEF94FF46020CDE912048DF84540A9
:1027E000012004278DF8440010948DF8507010A932
:1027F0003046FEF74DFA01231A4605213046FEF712
:1028000098FA0123022206213046FEF792FA0123AC
:10281000032207213046FEF78CFA012304220F2100
:102820003046FEF786FA484600F0A2F901A800F00B
:1028300042FA8348854D4C30CDE90254019004970B
:102840008020CDE9054040000790800008902020BE
:1028500009904FF44050CDE90A0401A9484600F020
:102860000DFA01213046FEF75FF80121484600F0DD
:1028700073F901213046FEF74DF847F230501594B8
:102880001599491C15918142FAD301213046FEF772
:102890008FFAADF8004040F2DC584FF40077B346B1
:1028A0001FE0404615941599491C15918142FAD3B1
:1028B00029880D9808440D9068880E9908440E9058
:1028C000A8880F9908440F90E8880C9908440C9048
:1028D00001215846FEF76CFABDF80000401CADF827
:1028E0000000BDF80000B842DBD358490D9808310C
:1028F000C01108830E98A1F11004C01148830F98ED
:10290000DFF84CA1C01188830C98524BC01188800D
:102910006068BAF9005040F6B4120580BAF902C0F6
:10292000A0F802C0BAF904708780BAF90660C680C0
:102930009AF80180B8F1FF0F21D0A5F5D854263CB4
:1029400094420FD2ACF5D05CACF5937C944509D29F
:10295000A7F5D857263F974204D2A6F5D856263E6B
:10296000964204D3D88840F48040D8803BE00D8361
:1029700042884A8382888A83C088888033E0B1F99C
:102980000450A5F5D855263D954214D2B1F91850FA
:10299000A5F5D855263D95420DD2B1F91A50A5F5A9
:1029A000D855263D954206D2B1F91C50A5F5D8550B
:1029B000263D954203D3DA8842F48042DA80DA88F1
:1029C000520410D40A8B02804A8B42808A8B828008
:1029D0008988C1805546504600F0CCFB0822284625
:1029E000616800F0DDFB00215C465846FDF79CFF66
:1029F00000214D46484600F0AFF800212046FDF783
:102A000089FF104E00213046FDF784FF0220C102ED
:102A1000401C8842FCD32046FEF7A8F83046FEF75B
:102A2000A5F8284600F0A4F8FDF788FF0A493C20E5
:102A3000087062B617B0BDE8F08F000000100240C9
:102A400000240140002801400800024050050020F9
:102A500000700308480C00206C07002010B5FEF73A
:102A6000BFF9C8214843800B10BD000070B5204B52
:102A700040F6C81441F2B7055B6C48F6E6065C43C5
:102A800005EBA4341B4D73434EF6F61606EBA33349
:102A9000C5E90443D460401A5361106091688842CC
:102AA00002DA4942884200DC116010684343107E1C
:102AB0000341906A19189162506A814200DD906268
:102AC000916A106A814201DB084600E09062A861C9
:102AD00011684C43117C0C4108412118B2F91C00CB
:102AE000884204DBB2F91A00884200DC08B270BDEB
:102AF000500100202801002010B54FF4005420465A
:102B000000F0ACF8002813D00A49087840F008001B
:102B10000870204600F014F80021074800F01CF867
:102B20000648C17E012903D10021C1760121017728
:102B300010BD0000B206002044000240500D0020ED
:102B4000C10002D5024908607047024948607047D9
:102B500004040240000002400029016802D041F054
:102B6000010102E04FF6FE72114001607047000063
:102B700001684FF6FE721140016000210160416062
:102B80008160C1603149314A0839904203D14868B7
:102B900040F00F0006E02D4A1432904204D14868FC
:102BA00040F0F00048607047284A2832904203D134
:102BB000486840F47060F5E7244A3C32904203D103
:102BC000486840F47040EDE7204A5032904203D10B
:102BD000486840F47020E5E71C4A6432904203D113
:102BE000486840F47000DDE7184A7832904203D11B
:102BF000486840F07060D5E7154A111F904203D134
:102C0000086840F00F0006E0114A1432904204D1E7
:102C1000086840F0F000086070470D4A2832904282
:102C200003D1086840F47060F5E7094A3C329042ED
:102C300003D1086840F47040EDE7054A50329042F5
:102C4000EAD1086840F47020E5E70000080002407F
:102C500008040240406880B270470000014600202E
:102C6000CA0001D5034A00E0034A12680A4200D0B4
:102C700001207047000402400000024030B50368A4
:102C800047F6F07293430C6A8A682243D1E90445FF
:102C90002C4322438C692243CC6922434C6A224351
:102CA0008C6A22431A430260CA6842600A688260E2
:102CB0004968C16030BD0021016041608160C16030
:102CC000016141618161C16101624162816270475C
:102CD00010B5114C8CB000212046FFF73DFF204677
:102CE000FFF746FF0D4800900D480021CDE9010196
:102CF0006420CDE903018020CDE905010791089109
:102D000009910A9169462046FFF7B8FF0121204644
:102D1000FFF722FF0CB010BD5800024004380140FC
:102D200030090020F0B540F6AA222A49C284838BDC
:102D30000C88E31A9BB20F2B0DD309888183037E85
:102D400000213BB1244BB3F90A40244B062C03DA93
:102D5000818429E08184F0BD214C2478022C02D0AA
:102D6000002CF5D0F0BD1F4C40F68B27656C1B4C3A
:102D7000A5F22D16BE42B4F9004017D2418B491C72
:102D800089B241836429EDD364214183B0F92410D1
:102D9000914201DA01EB22128284641C20B24FF4CA
:102DA000007118808842DDDB1980F0BD41F2941675
:102DB000B542FADBB0F92450002D02DDA5EB22125A
:102DC00000E0002282844183641E20B21880002823
:102DD000EADDF0BD780700206000002070040020CC
:102DE0006F0700205001002010B50446B0F9020022
:102DF00043F6991148438113E06840F266625043FC
:102E000001EBA030E060B4F9001043F69912514391
:102E10008A13216940F26663594302EBA1312161B3
:102E200006F096F86061A18840F6AB220844401095
:102E3000A0F515415539E062914205D9A0F5F85148
:102E4000FF39521C91421DD249F25451884202DD91
:102E5000A0F5204002E0A0F5F850FF38206300EB19
:102E6000400040F34F002085B4F924104A429042BC
:102E700001DA104602E0884200DD0846E083228441
:102E800061848AE0A0F5FE42FF3A41F255518A4240
:102E900014D8A2F6AA20206300EB400040F34F00B4
:102EA0002085B4F924205142E183884201DA0846A2
:102EB00002E0904200DD1046404250E0A0F5D442CE
:102EC000AA3A8A4215D2A2F6AA20206300EB40005B
:102ED00040F34F012185B4F924004242E28320846B
:102EE000914201DA104602E0814200DC084660842B
:102EF00053E0A0F5AA42543A41F256539A4215D2F1
:102F0000A2F6AB20206300EB400040F34F00208589
:102F1000B4F924104A42904201DA104602E0884295
:102F200000DD08464042E083218419E0A0F580429C
:102F300041F254539A4215D2A2F6AA20206300EB24
:102F4000400040F34F002085B4F92410E1834A4249
:102F5000904201DA104602E0884200DD08462084F3
:102F600062841AE0A0F52852AB3A8A4215D2A2F642
:102F7000AA20206300EB400040F34F012185B4F903
:102F80002400E08342422284914201DA104602E0AA
:102F9000814200DC08464042A9E7B4F91E004142E4
:102FA0000948B0F9000041438913E180B4F92010C9
:102FB0004942414389132181B4F9221049424143D6
:102FC0008813608110BD000070040020012101768B
:102FD000704770471548164A4FF48041007804281E
:102FE00021D002F13C03D08A9B88C01A00B22F285E
:102FF00001DD001108E0002801DD002007E00D4B95
:10300000984201DA184602E0402800DD402093890A
:10301000184400B2884203DC40F26661884200DA5C
:103020000846908170479181704700006F0700202B
:10303000EC040020C0FEFFFF38B54B484B49028826
:103040000B889A1A92B20F2A71D30988484C0180D2
:103050004FF0FF01E2884FF47A7355044FF49670F5
:1030600002D51622009103E0950403D515220091A4
:10307000014670E0D50402D514220091F8E7150549
:1030800002D513220091F3E7550502D512220091D3
:10309000EEE7950502D511220091E9E7D50502D5A5
:1030A00010220091E4E7150602D50F220091DFE718
:1030B000550602D50E220091DAE7950602D50D22BB
:1030C0000091D5E7D50602D50C220091D0E715076F
:1030D00002D50B220091CBE7550702D50A220091B9
:1030E000C6E7950702D509220091C1E7D20702D0B1
:1030F00008220091BCE76289550702D5072200919A
:10310000B6E7950702D506220091B1E7D20702D0B3
:1031100005220091ACE7227BD20702D00422009165
:10312000A6E7E289D40603D503220091A0E719E0BF
:10313000140702D5022200919AE7540703D494079A
:1031400001D4D20702D00122009191E7002003466A
:1031500002460146009003F0B1FFBDE83840024846
:10316000FDF728BF38BD00003C0C00207807002088
:10317000480C002070B50546002472B600F0FEF839
:10318000252000F073F8284600F076F8042801D0D6
:103190004FF0FF3400F0A4F862B6204670BD000086
:1031A0002DE9F04700251746894680462C4672B621
:1031B00000F0E4F812E000BF59F82460352000F078
:1031C00055F83146404600F0AFF8042802D04FF0E1
:1031D000FF3506E0641C08F10408E4B2B4EB970F75
:1031E000EAD300F07DF862B62846BDE8F08700001B
:1031F00070B51148114C4FF00005C088810503D40B
:10320000410601D4C00515D54FF480610C4800F08B
:1032100049FB68B9A08840F6B831884201D2401C09
:10322000A08080B2B0F57A7F01D30120607070BDBC
:10323000A58070BD6570FBE7480C0020900700205A
:10324000000C0140084946F668000880091D088006
:10325000091D41F6DD5008800348001F018841F038
:103260002001018070470000182C01400149C8600E
:10327000704700000020024070B50D4E05463046F4
:1032800000F088F8042811D10A4C206940F00200AF
:1032900020616561206940F040002061304600F007
:1032A00079F8216941F6FD721140216170BD00007D
:1032B000FFFF0F000020024008490420CA68D2071F
:1032C00001D001207047CA68520701D5022070471B
:1032D000C968C906FBD503207047000000200240E2
:1032E0000248016941F080010161704700200240FD
:1032F000F0B506464FF6FF770D46384600F04AF81F
:1033000004280DD1074C206940F001002061358070
:10331000384600F03FF8216941F6FE721140216104
:10332000F0BD0000002002402DE9F84106460020D3
:103330004FF6FF7700900D46384600F02BF8042832
:1033400017D10D4C206940F0010020613580B8464E
:10335000384600F01FF841F6FE77042806D1B61C67
:10336000280C00963080404600F014F8216939405E
:103370002161BDE8F88100000020024003480249B5
:1033800041600349416070472301674500200240C6
:10339000AB89EFCD00B50346FFF78EFF03E000BF1A
:1033A000FFF78AFF5B1E012803D0002B00D1052008
:1033B00000BD002BF4D1FAE710B5C28800210AB194
:1033C000032206E042890AB1022202E0828912B198
:1033D0000122027000E0017004784FF4804344F64B
:1033E000206244B1012C06D0022C07D0032C01D15D
:1033F0004180818010BD4380828010BD41F2333115
:10340000418040F6B731F4E7401A10609168884275
:1034100002DA4942884200DC116051691068137E6B
:1034200041431941936A0B449362516A8B4200DD18
:103430009162936A116A8B4200DA9162D168936A51
:103440004143107C01410341B2F91C0019448842F8
:1034500004DBB2F91A00884200DC08B270470000B1
:10346000054920B1086940F08000086170470348B1
:1034700048600348486070470020024023016745C8
:10348000AB89EFCD06494FF47A70CA68D20705D0F0
:10349000401E0004000CF8D1FF2070470020704748
:1034A000002002400E4A0320A2F1580182F83E009B
:1034B000002088810B490886C862C8830884488434
:1034C00090620948016DB1F5206F01DBA321916283
:1034D000807A002802D0906A4042906270470000D3
:1034E0006000002058050020500100200C490020F9
:1034F000A1F15802488108811082D081A1F86000B2
:1035000048668866A1F874009080508010809061B1
:10351000044A9062303A906281F85E00FFF750B83A
:1035200060000020480A0020F0B53D4988894A899A
:10353000801A80B20F286AD388894881CA8939489D
:103540000B3A272A26D28A7822BB8268384B42F46B
:1035500080728260344A374C374D12785607334AAE
:103560000AD4364E36881680354A12881A80354A73
:1035700012882280344A09E0344E36881680344A54
:1035800012881A80334A12882280334A12882A808D
:1035900001228A70314A0021314B82F84D101946C0
:1035A0009A7F304D0968802A32D302F01F0255F805
:1035B000222011422CD0826822F48012184E8260A0
:1035C000123614461215B778521C62F38617264A33
:1035D000B77093F816C01778BCF1800F27F0020679
:1035E00008D30CF01F0C55F82CC011EA0C0F01D1B8
:1035F00047F0020616701A7E802A0DD302F01F02D1
:1036000055F82220114207D144F400218160F0BD19
:10361000826842F48012D1E724F40021F6E700002A
:103620006C070020C002002050010020E4040020AC
:10363000E6040020E8040020EA040020D40400206E
:10364000D6040020D8040020DA040020DC04002086
:10365000DE040020E0040020E2040020A40E00208C
:1036600018060020B8C10008EC04002070B52148FD
:1036700081890289891A89B20F2932D381891E4D25
:103680001E4C0181697A22681D4E42F00400802997
:1036900008D301F01F012B6856F821100B4201D10D
:1036A00022F004002060FFF7A3FDA87B802819D337
:1036B00000F01F00296856F82000014212D120684E
:1036C00020F002002060E87A80280FD300F01F006D
:1036D000296856F82000014208D1206820F008002F
:1036E000206070BD206840F00200EBE7206840F0E9
:1036F0000800F5E76C07002018060020C002002033
:10370000B8C1000830B5044600204FF4004302461B
:1037100040EA030101FB01F5A54200D80846521C0E
:103720005B0812B2102AF3DB30BD0000F0B51D4C6F
:103730001B4A4FF0010C94F83B5094F80AE01446F1
:1037400092F83C3094F838402B43651CEEB2154D8E
:1037500095F83D700025BEF1FF0F0AD0BEF1000FB5
:1037600006D18B4213D155700C2C01D282F83860EF
:10377000F0BD834202D182F801C0F5E78B42F7D158
:103780005570B80709E000BF82F83850F0BD834299
:10379000FCD1F84382F801C080070028F4D0F0BDC6
:1037A0007404002050010020F0B5CA78002502F012
:1037B0000F03D20601D58A7813430A784FF00F0E13
:1037C00012F0FF0F4FF001021CD004680F8802FABC
:1037D00005F63740B74211D14FEA850C0EFA0CF7C7
:1037E00024EA070703FA0CF43C43CF78282F02D0D1
:1037F000482F02D002E0466100E006616D1C082DF2
:10380000E4D304600C88FF2C1ED944685FF00006E6
:1038100006F1080702FA07F50F882F40AF420FD1D3
:103820004FEA860C0EFA0CF7BC4303FA0CF73C4344
:10383000CF78282F00D14561CF78482F00D105617E
:10384000761C082EE4D34460F0BD0000F0B5144CA3
:10385000002801DAE36900E06368420D120185B2D5
:10386000C0F301579540C0F30346032F05D0C202B1
:103870000AD50322B240934307E023F070626368E5
:1038800023F07063636002E0AB4343F0706201B108
:103890002A43002801DAE261F0BD6260F0BD000059
:1038A000000001400246002092680A4200D0012038
:1038B000704741617047016170470AB1016170470B
:1038C000416170474FF6FF62B0F57F4F04D0911C05
:1038D000884203D100207047104670470449098888
:1038E000814201D3081A01E0101A084480B27047DF
:1038F000C80800200148008870470000C808002060
:103900000F4A104B92F838105B5C834201D10120C2
:1039100004E00D4B5B5C834203D1002082F83A0047
:1039200070470A4B5B5C834201D18120F6E7084B6C
:10393000595C814201D18020F0E70320EEE70000CE
:103940005001002070C6000882C6000876C6000834
:1039500088C600080A4810B501784FF000024C07ED
:1039600008494FF0FF0389684FEA017105D5002926
:1039700001DA827210BD837210BD0029FBDBF8E70B
:1039800050010020C0020020F0B5194E194C002251
:10399000E31CA6F1060CB75CA518ED78FF5C0D439F
:1039A0000F43BD421FD01CF80270FF5C0F43BD42A5
:1039B00019D015460023A618F6780E43C6545B1C92
:1039C0001CF80220DBB2062BF5D3C1788170017997
:1039D000C17000214218491C15711CF80550C9B26C
:1039E0000629F7D3F0BD521CD2B2032AD3D3F0BDBF
:1039F0004ABD00087404002010B502460021064BA1
:103A000006205C186478944200D10846491CC9B26B
:103A10000629F6D310BD0000500100200548D0E96A
:103A200000218A4202D14FF0FF30704700EB0110B5
:103A300080687047EC10002070B5164C05464FF0BA
:103A4000FF36D4E90010814221D004EB00108068D9
:103A50006860606804EB0010007B00F00F02AA723F
:103A600004202872606804EB001105F10B000E3190
:103A7000FCF789FB72B66068401C6060402801D387
:103A80000020606062B6A87A08B1002070BD3046A0
:103A900070BD0000EC100020F0B52D484FF0000282
:103AA0008078C1072B484ED02B494FF4FA6CA0F117
:103AB0003807B1F904502949B1F8763095BB496C03
:103AC00061452FDD90F84A1061B32549C9790C068C
:103AD00028D501F07F015A2924D290F82B11491CD6
:103AE000C9B280F82B11C8291CD380F82B21D0F83B
:103AF0003041014604F11E0691F82C11B34203DD5A
:103B0000052908D2491C01E041B1491E80F82C1159
:103B1000C9B2052902D3012180F82A11191B396382
:103B2000C0F830310F490978C90702D10DB9634592
:103B300008D280F82A2180F82C2180F82B21C0F8A7
:103B400030313A63F0BD80F82A2180F82C21F0BD95
:103B5000BF070020C00200201006002050010020F6
:103B6000DF070020F80A00204FF42032C260002155
:103B700081620E22028241F26202426108220283C5
:103B80004FF46042428381834FF07842C0E90821BC
:103B900040F6C41101807047B0F90010B0F902205E
:103BA000891A41604269037E4A431A41836A134479
:103BB0008362426A934200DD8262836A026A9342B0
:103BC00000DA8262C268836A4A43017C0A410B417F
:103BD000D118B0F91C208A4201DA10467047B0F9BA
:103BE0001A008842FADC08B27047000010B5144889
:103BF0001449B0F894200B889A1A92B2B2F5437F18
:103C00001DD90988A0F89410B0F8921020F8601F10
:103C1000002242860C480D4CC2888280C180C38934
:103C200083812489891AA4B2C4818160E11A016167
:103C3000074A818AC182928A8282511A816110BDAB
:103C400050010020780700206C0E0020580500204D
:103C50006000002009480A49B0F8B2200B889A1A7F
:103C600092B241F684639A4206D3098820F8B21FC3
:103C70004188818000214180704700005001002070
:103C800078070020134930B4087AC0071FD11248C2
:103C9000CC880278630606D4930604D4530602D473
:103CA00090F83B3003B1012324F04004CC8022F093
:103CB00060010170002180F83B102BB1074800F82B
:103CC0005E1F41804176017630BC00F06FBB30BC96
:103CD00070470000480C00205001002060000020C8
:103CE0000D480178C90702D00C49098801E04FF658
:103CF000FA714166094901201039088007482438C3
:103D0000018841F00101018004481838018821F040
:103D10001801018070470000500100202404004079
:103D20000A49D1F8982012B1521EC1F8982031F8F2
:103D3000922F521C21F81A294A6A521C4A628A8F11
:103D4000521C8A8701F8400C704700005001002087
:103D50002DE9F041274827498079B1F808C040068D
:103D600002D45FEACC7035D02348244B2449007834
:103D70001C785FEA406E2348CB7B1F4990F85E5069
:103D8000428F496C4FF0040640F6C41702D55FEA33
:103D9000CC7C04D0042D14D0022C1DD018E0042DAE
:103DA00002D0022C10D013E040F69803994208DCB0
:103DB000002100F85E1F41804176017620F84E2CEC
:103DC00007E000F055F804E0022B01D1B94207DC0E
:103DD00002820120BDE8F081022BF9D1B94202DD57
:103DE00080F85E60EDE78229F2DC07490978090670
:103DF000EED5E6E7480C0020500100206F070020B8
:103E0000C002002060000020400700201349087A0B
:103E1000C207134805D18979490615D501784906A5
:103E200012D4104991F85E10042905D0406C40F678
:103E3000C411884208DC09E00B4840F2DC51806E76
:103E4000884201DA0120704700207047074909784D
:103E50000906F7D58228F7DDF4E70000480C0020BA
:103E6000500100206000002094090020400700203D
:103E70002DE9F0478D4C94F85EC0BCF1010F08D0DD
:103E8000BCF1020F05D0BCF1030F02D0BCF1050F4D
:103E90000BD187480078022803D18648C07B0228CE
:103EA00003D0BDE8F047FFF721BBB4F8600010B1C4
:103EB000401EA4F860007D4D7F4F583D0323E889E4
:103EC000298A02B20026DFF8F4A1F86C4FF001094C
:103ED00009B2BCF1060F0BD2DFE80CF0030C1C3169
:103EE000E28BFEF76DFB268166816E8084F85E9022
:103EF000BDE8F087FFF7A6F940F266602882EE8100
:103F000026826E80022084F85E0043F69820A4F892
:103F10006000EDE761812281B4F860000028E7D1FC
:103F200084F85E304FF48030C4E9196064488662DA
:103F300030388662A4F86C606E802667D8E76181AD
:103F40002281B4F860004FF0050830BBA4F860800F
:103F5000A888401C80B2A880022808D90123022228
:103F600042F6CC4003F0B6F82882EE81AE80B4F879
:103F7000660058B3A4F86690D4E919100844A06606
:103F8000B4F86A1040F28270814201D3A4F86A004A
:103F9000208AB4F86A10401A2082B7F84C0081B227
:103FA000208AFCF728FF00B2A4F8740044F61F61D1
:103FB0000844490088421AD8B96D514517DC688811
:103FC000B0F5FA7F06D2401C688091E7606E401C15
:103FD0006066D1E7B4F86A10B1FBF8F14942A96113
:103FE0002E806E80A4F8606084F85E8080E76E802A
:103FF0007EE761812281B96DD046414506DD2E8084
:104000006E80A4F8606084F85E3071E70A2291FB4C
:10401000F2F2A969531E994201DA491C03E0531CCC
:10402000994202DD491EA96100E0AA61218A2A8B1A
:1040300080B2114489B22182FCF7DDFEC11700EB8A
:1040400011610912042901DD042104E06FF003026B
:10405000914200DA1146228A114421824142A4F899
:104060007410002800DA0846B0F57A7F16DAB96DC8
:10407000414513DC29884FF49672914204D2491CC1
:1040800089B229809142A0D3B7F84C002082A4F8CD
:104090006060042084F85E002E80A8E72E8027E769
:1040A000208284F8779084F8766021E76000002011
:1040B0006F070020C00200209409002048F4FFFF91
:1040C000480A002070B53C4D4FF480712846FFF738
:1040D000E9FB840080212846FFF7E4FB44EA400422
:1040E00040212846FFF7DEFB34490443E3B291F850
:1040F00078209A425FD05A4081F87830012A03D064
:10410000022A01D0042A56D181F8542081F87B205C
:1041100091F87C00294C9043083C81F87C0062783F
:10412000FF2A01D2521C627091F87A2001259D402D
:104130002A4209D12A4381F87A2091F87920FF2A6E
:1041400002D2521C81F8792091F879501C4A1D4BFB
:10415000042D06D320B3012825D0022823D004281B
:1041600021D06478062C26D3032803D0052801D05B
:10417000062820D1D48844F04004D4800A7822F064
:10418000400242F020020A7081F83B00187840F0AB
:104190008000187000F00AF9BDE8704000F076B8B1
:1041A000FFF770FDF8E7D48844F04004D4800A7823
:1041B00042F06002E7E770BD0010014050010020AE
:1041C000480C0020400700201CB52D4890F83B30DB
:1041D00090F83C20934252D000248DF80440534084
:1041E0008DF800309DF800300122012B08D09DF899
:1041F0000030022B09D09DF80030042B0AD00DE0CE
:104200001F498DF80420443108E01D498DF8042031
:10421000463103E01A498DF8042048319DF8042006
:10422000012A2CD190F83D309DF80040154AA34258
:1042300017D090F83E309DF80040234208D0B0F8E7
:104240004C30A0F84A300B881488E31AA0F84C30A0
:1042500090F838302BB1B0F840301488E31AA0F849
:10426000423012880A80A0F8402010F83E1F9DF8C6
:104270000020114300F801199DF8001001701CBDC9
:104280007404002078070020FFF71CBF70B50F4DA5
:104290004FF480712846FFF705FB840080212846F3
:1042A000FFF700FB44EA400440212846FFF7FAFAF2
:1042B00004430748072100F8784F0171002141703D
:1042C0008170C17002480838417070BD0010014013
:1042D0005001002070B5344890F83A10CA43920754
:1042E00061D001F0030280F8392090F83D305B0680
:1042F0001B0E80F83D30012A01D0812A02D15B1CBF
:1043000080F83D300278D2074DD0DBB203F00102D5
:10431000C3F34004A24246D1B0F856400025641CC5
:10432000A0F85640204CA0F8585090F83E60A47A6F
:10433000B24202D080F83E200DE0A607B6EB837FA4
:1043400002D080F83F5006E090F83F30642B02D254
:104350005B1C80F83F3090F84030642B0CD25B1C23
:10436000DBB280F84030022B06D204F00103934206
:1043700002D1022280F84020012901D0002912D167
:1043800090F83820416E00EB820291610163D0E920
:1043900006121144D0E908231A441144826A1144D8
:1043A000C26A1144416370BD50010020064890F874
:1043B0003B10064890F82720914204D080F827103F
:1043C000034920200870704750010020A40E0020EF
:1043D0006C070020FEE700002DE9F04F00BF002031
:1043E0009E4E9F4AA6F51271A6F5BE79A6F1440B22
:1043F00006F1440E804601F5E074A1F1780301F561
:10440000457A1D5C15F0C00706D0402F51D0C02F53
:1044100077D0802F76D004E115F01F0504D0154425
:1044200040F080072F7201E082F80880012826D032
:10443000022824D0032822D0042820D008281ED007
:1044400010281CD0874D55F820C0DCF8005054F8D7
:1044500020703D40CCF80050824D55F820C0DCF86B
:10446000005056F820703D43CCF800501D5CAD065E
:1044700059F820502F6813D53AF810C03EE051F893
:1044800020502F6854F820C007EA0C072F6051F81D
:1044900020502F6856F820C047EA0C072F60E5E748
:1044A000DFF8B8C10CF1F00C5CF820C007EA0C078B
:1044B0007EE015F01F0504D0154440F080072F72F0
:1044C00001E082F8088001281DD002281BD00328B3
:1044D00019D0042817D0082815D0102813D0614D02
:1044E00055F820502F6854F820C007EA0C072F60B9
:1044F0005C4D55F820502F685BF820C047EA0C0748
:1045000056E00BE056E051F820502F6854F820C0D8
:1045100007EA0C072F6051F82050ECE715F01F0553
:1045200005D0154440F0800785F8217001E082F83D
:104530002180012825D0022823D0032821D0042857
:104540001FD008281DD010281BD0464D55F820C07C
:10455000DCF8005054F820703D40CCF80050414D3C
:1045600055F820C0DCF800505EF820703D43CCF8D0
:1045700000501D5CAD0615D53A4D3AF81070CC359B
:1045800014E051F820502F6854F820C007EA0C07B7
:104590002F6051F820502F685EF820C047EA0C07C2
:1045A0002F60E6E72D4D3AF81070E03D55F82050A9
:1045B0002F6036E015F01F0505D0154440F0800748
:1045C00085F8217001E082F82180012830D002288E
:1045D0002ED003282CD004282AD0082828D0102830
:1045E00026D0204D55F820C0DCF8005054F820703B
:1045F0003D40CCF800501B4D55F820C0DCF8005071
:10460000164F883757F820703D43CCF800501D5C9A
:10461000AD06B1D4114F3AF81050E03F57F8207072
:104620003D60401CC0B21128FFF4EBAEBDE8F08F36
:1046300051F820502F6854F820C007EA0C072F606B
:1046400051F820502F68DFF814C00CF1880C5CF88A
:1046500020C047EA0C072F60D9E7000044C40008D7
:104660001806002040C200084FF40771C1824FF4C1
:104670005861018340F6145181837047F0B5C48AB4
:10468000B0F900608681B0F90250C581B0F90430FC
:104690000227002101220382AB4204DBB54202DD86
:1046A000C78042810CE0B34204DBAE4202DDC7802A
:1046B00041811CE09D4205DBB34203DDC28047819E
:1046C000018115E0B54204DB9E4202DDC2804181DA
:1046D00005E0AE4205DB9D4203DDC18042810781DA
:1046E00006E09E4204DBAB4202DDC18047810281CD
:1046F000C388458900EB430700EB4505BB89AE89BC
:104700009B1B0FFA83FEA0F812E00689AB8900EB31
:10471000460CBCF80CC0A3EB0C038382B0F9183034
:10472000B7F90CC0A3EB0C0CB4EB4C0F04DA80F817
:104730002010A3F1A10113E0A64503DD80F82010AD
:10474000B9890BE026B1012E04D0022E10D004E06E
:10475000062100E0052180F82010A989091B6D3190
:10476000418309B2B1F5586F04DB5B1E438304E05B
:104770000421F0E7002900DC4283418B8183F0BDF6
:104780000B49002288760A62CA614A62094A32F9F4
:10479000103002EB40028B62B2F90220CA62064A74
:1047A00032F810000882A1F86000A1F8620070479A
:1047B000080200209AC600088EC600082DE9F05FA6
:1047C000FE48FF4982880B889A1A92B20F2A47D373
:1047D00009888180FB498346FB4D0888FB4FDFF841
:1047E000F0934FF00108002678B3401E0880EE7366
:1047F000EE6249462868B1F90210430742F6AA2240
:1048000018D4FB8843F40053FB8099F800309B07D1
:1048100009D5AB6823F08003AB60A5F8806085F80C
:10482000826085F88360C30404D485F8F480C5F8F9
:10483000F06003E085F8F460430707D4914205DB9C
:1048400085F8F880A5F8F66004E010E085F8F860D7
:10485000430703D4914201DBC00703D085F81561FB
:10486000BDE8F09F85F81581A5F81661F8E7B5F861
:104870001C0143F69821884202D2401CA5F81C0175
:1048800002F032FCDFF84CA39AF8500010B1FDF7AB
:10489000C1FE05E0C9481838017821F00101017016
:1048A000FFF7FAF800F024FACB4841F26802416CB5
:1048B0004FF40060914201DBC84A04E0B1F57A6F21
:1048C00002DAC64A121D10609AF85100D446DFF889
:1048D000F8A20A24C007AAF1380A38D0C048807B61
:1048E000802802D32878800705D5BE480078C20604
:1048F00001D4800627D5EA7B8AF8092099F8003090
:10490000AE4A23F00203183A89F800305680137833
:10491000504623F001031370BA7952060FD4C289AE
:10492000B2F5FA7F03D2521CAAF80E200FE040F62F
:104930003C70814201DD002466E0042464E0002430
:10494000AAF80E6060E08AF80560AAF80E60A86810
:10495000020501D5082457E09CF83FE05FEACE72DB
:1049600047D0DFF87CC2EA7B8AF809209CF809303E
:10497000802B43D39C4B9B781B063FD52B785B0742
:1049800030D4FB889B0403D520F02000A86030E0E1
:104990008A4B40F02000183B5E801C7824F0010414
:1049A0001C70A8609CF8170080280BD300F07F04CF
:1049B0004FF00040DCF80030E040034202D185F8BF
:1049C000048000E02E712879C00702D15FEA8E7062
:1049D00005D50324032A17D08AF80C8014E000249C
:1049E000EE6211E020F02000A860F88820F400506A
:1049F000F88095F82A01012805D005E02A6842F0E0
:104A000004022A60C0E7092408B2784903F05AFD7D
:104A10006D49774DCA6A50438013A1F8E8000A2C0B
:104A200070D171488078800602D5FCF75BFA09E006
:104A300065488168CA0502D521F0080101E041F00E
:104A40000801816060484FF400535A0090F84AC052
:104A500042F2666E42F6CC41BCF1010F17D0BCF1B8
:104A6000020F26D0BCF1030F95F800C0614945F64E
:104A70009444CCF3810C07D043F6FE78BCF1010FCF
:104A80003DD0BCF1020F3AD0A0F8182120E02C78DC
:104A9000C4F38104012C06D0022C07D0A0F8181111
:104AA000A0F8481017E0A0F818E1F9E7A0F81831CD
:104AB000F6E72C78C4F38104012C06D0022C04D034
:104AC000A0F81821A0F8482005E0A0F81811F9E78F
:104AD000A0F848200C8044498978490708D52978EE
:104AE000C1F3810101290ED0A0F81831A0F8483097
:104AF000324918390B78DB0708D00B8A08E0A0F898
:104B00001881E5E743E0A0F818E1EFE7B9F80430D1
:104B1000ABF8123019B2B0F948305943C1F38F33B2
:104B20005146AAF81E30934200D9CA83324A1278FD
:104B3000D20605D5CB8B41F23332934200D2CA83E1
:104B40008268C2F3C003C2F30024A34205D1CC8B18
:104B500041F699139C4200D9CB83284B9B78DB0705
:104B60000AD0D20108D41F4A137803F00F03032B95
:104B700002D19279920700D0CE83BAF81E10C1629A
:104B8000002903DD1E480224067000E000249BF883
:104B90001A0090B9022C40D07CB10F4803789906D6
:104BA00033D5B979490630D590F83B1001293BD06F
:104BB000022939D0042937D024E03FE0100B00202F
:104BC000780700207A070020C0020020480C00204F
:104BD00010060020A40E002050010020100C0140FF
:104BE00018060020DF070020BF07002094BC000843
:104BF000EC0400204601002040070020AF07002001
:104C00008C07002023F040010170F88820F4006038
:104C1000F880B9F8041051B10CE0288F0028BCD1FD
:104C200043F698202887B8E743F04001ECE720F0EE
:104C30008000F88080B220F02000F8801448406C9A
:104C40004E281FDBFB8818061CD5BAF81C104FF441
:104C5000FA75491C89B25046AAF81C10A94201D91C
:104C6000858301E0A94207D3B9F8041021B9AAF855
:104C70001C6023F08000F88099F8001021F00201F8
:104C800089F8001003488BF81A40C473E8E5000067
:104C900050010020C002002070B500230C8863F38F
:104CA0000F02012505FA03F6344206D0C3F10F06C0
:104CB00005FA06F1114361F30F025B1C102BF1DBC7
:104CC000028070BD70B500230C7863F307020125E4
:104CD00005FA03F6344206D0C3F1070605FA06F1D9
:104CE000114361F307025B1C082BF1DB027070BDFE
:104CF000F0B5204890F866101F480129836823F416
:104D0000006234D11D49CE88740630D41C4D1F0575
:104D10004FF00004B5F9025020D41A4A526C642AAC
:104D200011DC40F6386295420DDAB2040BD40278F9
:104D3000520710D4B0F8D82040F6B835AA4203D2B2
:104D4000521CA0F8D820F0BD43F400628260D0016C
:104D5000F9D48C81F0BDA0F8D840F0BD41F2CD036C
:104D60009D42FADD097BC907F7D18260F3E78260D3
:104D7000F0BD0000A40E0020C0020020480C00205E
:104D80001006002050010020F0B5364D364F044685
:104D900095F83B0097F83B1023780843EE1C6278A7
:104DA000834205D1E0781146FEF7C0FC207908E087
:104DB00094F802C084450CD1E1781046FEF7B6FCA9
:104DC000E07905F82F0F2878805D6870287BE877F8
:104DD000F0BD82421DD161461846FEF7A7FC95F84A
:104DE0004E1095F83B00814207D1B97A09B1A179FB
:104DF00000E0617985F82F101EE06978012901D063
:104E0000A17922E0617927E0297841F00401297035
:104E100012E0E1788142DBD119466046FEF786FC5C
:104E200095F84E1095F83B0081420AD1B97A09B144
:104E3000617ADFE7217ADDE715F82F1F895D697058
:104E4000C5E76978012906D0617A85F82F10B97A0B
:104E50000029F1D1D8E7217A85F82F10B97A0029F5
:104E6000EAD0D1E774040020500100200B480178FB
:104E700021F0020100F8381B002100F818194177D1
:104E8000817733218185418508214184012100F802
:104E90001F1C034880F8391070470000740400207C
:104EA000500100200D4900B50B4851F8012F40F882
:104EB000032F89888180084801210930FEF764FDAD
:104EC000054802211330FEF75FFD034804211D3021
:104ED0005DF804EBFEF758BD74040020500100207B
:104EE000094944F648000880091D46F64800088034
:104EF000091D41F2111008800348001F018841F08C
:104F00002001018070470000182C01402DE9F0417C
:104F1000654C664B0025A0780126644A10330528AD
:104F20007ED2DFE800F00313113E1100108820F05C
:104F3000010010801D805E480580001F0580001F55
:104F40000580FFF7CDFFA670BDE8F081584941F616
:104F5000CC401C390880564945F658002439088051
:104F6000091D46F65800088051492020283908803C
:104F70000020401CC0B27328FBD3FFF7B1FF4B49A0
:104F800084F85C502C3147F6906008804748143014
:104F900006801D80108840F0010010800220A07063
:104FA000D2E700215FF0010004EB410204EB400373
:104FB000B2F85020B3F850309A4200D20146401C5B
:104FC000C0B20628F0D33B48405C84F83900FFF7B4
:104FD0004DFF1D2000F046FE00F074F8364E3748B5
:104FE0004FF4807196F83B20012A04D0022A1AD08F
:104FF000042A2ED044E08046FEF754FC870080212E
:105000004046FEF74FFC47EA400740214046FEF786
:1050100049FC074347F0010084F83B00224800E0C8
:105020003AE009302AE08046FEF73CFC8700802108
:105030004046FEF737FC47EA400740214046FEF76E
:1050400031FC074347F0020084F83B001648133058
:1050500014E08046FEF726FC870080214046FEF7DC
:1050600021FC47EA400740214046FEF71BFC07436E
:1050700047F0040084F83B000B481D3003F090FD1E
:1050800094F82F0086F838001D2000F001FE04205F
:10509000A0700B48057057E7108820F001001080C1
:1050A0001D80A57050E70000740400200008004037
:1050B0003C2C014050BD0008500100200010014070
:1050C0006F0700202DE9F041354C14F82F0F354DB6
:1050D000E0724FF4807739462846FEF7E3FB8600FE
:1050E00080212846FEF7DEFB46EA4006402128469E
:1050F000FEF7D8FB0643207BF1B22F3C814215D04E
:1051000084F83C0039462846FEF7CCFB8600802117
:105110002846FEF7C7FB46EA400640212846FEF730
:10512000C1FB064384F83B60FFF74EF81E4D95F82F
:105130003B00012827D0022828D0042829D018486D
:1051400094F83B102730085C04F8300F14F801097C
:10515000FEF752FC04F82F09A87A00B10120607014
:1051600002F062F894F84E0094F83B10884206D0A2
:1051700094F83800062802D2401C84F8380084F8DD
:105180004E10BDE8F0810648093004E004481330B1
:1051900001E003481D30BDE8F041FFF7F5BD000018
:1051A000740400200010014050010020FF2801D9A4
:1051B000FF207047C0B2704770B5474991F8720040
:1051C000AA287FD191F8730055287BD1434D002048
:1051D0000A5C2A54401CC0B27428F9D3404E286996
:1051E000C6F80100A88AA6F80500D5F81600F060F8
:1051F000D5F81A003061D5F81E001235706103F041
:1052000051FC3849688A888103F066FC287D123D8C
:10521000C007307802D040F0040001E020F0040024
:10522000314930704FF480400861304C15F8280F38
:105230002F4984F82000688B6080A88BA080E88BC1
:10524000E080288C2081688C608195F8240081F8AA
:10525000D60015F8010C86F83B000020C6F89C002B
:10526000FFF720FE2348A98E0183E98E4183298F11
:10527000818395F84210283D012908D0022901D0E8
:10528000032909D0217821F00C01083107E02178A9
:1052900021F00C01091D02E0217841F00C01164AB1
:1052A00021700121918195F8701001290BD095F89A
:1052B0006D1059B101290CD04FF4805100E001E08C
:1052C000A0F8761070BD44F21C71F7E74FF400515E
:1052D000F4E741F25551F1E700FC0008A40E00206C
:1052E0005001002060000020440E0020EC0400204B
:1052F000C002002058050020480C002010B5FCF723
:1053000005FAFE48FE4AFF49007BC00703D08878B3
:1053100020F0010005E09078800703D0887840F005
:1053200001008870F8480B7803704B7843708B78D5
:105330008370CB78C3700B7903714B7943718B7990
:105340008371C979C171EF49083109780172ED495A
:10535000083149784172EB49083189788172E9490D
:105360000831C978C172E749083109790173E54903
:10537000083149794173E349083189798173E149F9
:105380000831C979C173DF49103109780174DD49E9
:10539000103149784174DB49103189788174D949D9
:1053A0001031C978C174D749103109790175D549CF
:1053B000103149794175D349103189798175D149C5
:1053C0001031C979C175CF4918310B7803764B7804
:1053D00043768B788376CB78C3760B7903774B79DA
:1053E00043778B798377C979C177C6490F390978B3
:1053F00080F82010C3490F39497880F82110C1493D
:105400000F39897880F82210BE490F39C97880F8A1
:105410002310BC490F39097980F82410B9490F3994
:10542000497980F82510B7490F39897980F8261015
:10543000B44920310B7880F828304B7880F8293037
:105440008B7880F82A30CB7880F82B300B7980F875
:105450002C304B7980F82D308B7980F82E30C9793B
:1054600080F82F1000F1D001097880F8301000F199
:10547000D001497880F8311000F1D001897880F8A6
:10548000321000F1D001C97880F8331000F1D0015A
:10549000097980F8341000F1D001497980F835108D
:1054A00000F1D001897980F8361000F1D001C97976
:1054B00080F8371000F1D001097A80F8381000F137
:1054C000D001497A80F8391000F1D001897A80F84A
:1054D0003A1000F1D001C97A80F83B1000F1D001F8
:1054E000097B80F83C1000F1D001497B80F83D1029
:1054F00000F1D001897B80F83E1000F1D001C97B1A
:1055000080F83F1000F1D001097C80F8401000F1D4
:10551000D001497C80F8411000F1D001897C80F8ED
:10552000421000F1D001C97C80F8431000F1D00195
:10553000097D80F8441000F1D001497D80F84510C4
:1055400000F1D001897D80F8461000F1D001C97DBD
:1055500080F8471000F1D001097E80F8481000F172
:10556000D001497E80F8491000F1D001897E80F891
:105570004A1000F1D001C97E80F84B1000F1D00133
:10558000097F80F84C1000F1D001497F80F84D1060
:1055900000F1D001897F80F84E1000F1D001C97F61
:1055A00080F84F1000F1F0010B7880F850304B7804
:1055B00080F851308B7880F85230CB7880F85330B7
:1055C0000B7980F854304B7980F855308B7980F81E
:1055D0005630CB7980F857300B7A80F858304B7AB8
:1055E00080F859308B7A80F85A30CB7A80F85B306B
:1055F0000B7B80F85C304B7B80F85D308B7B80F8D8
:105600005E30CB7B80F85F300B7C80F860304B7C69
:1056100080F861308B7C80F86230CB7C80F863301E
:105620000B7D80F864304B7D80F865308B7D80F891
:105630006630CB7D80F867300B7E80F868304B7E1B
:1056400080F869308B7E80F86A30CB7E80F86B30D2
:105650000B7F80F86C304B7F80F86D308B7F80F84B
:105660006E30C97F80F86F10264950310B7880F872
:1056700070304B7880F871308B7880F87230CB784E
:1056800080F873300B7980F874304B7980F875307E
:105690008B7980F87630C97980F87710117880F8A6
:1056A0008010517880F88110917801F0030180F822
:1056B0008210117980F88310517980F884109179E3
:1056C00080F88510D17980F88610117A80F88710DB
:1056D0000C4938310A7802F0030280F888204A78B1
:1056E00080F889208A7880F88A20CA7880F88B2010
:1056F0000A7980F88C204A7908E00000480C0020E4
:105700005C100020AF0700204C0F002080F88D2097
:105710008A7980F88E20C97980F88F106B490A78D1
:1057200080F890204A7880F891208A7880F892203A
:10573000CA7880F893200A7980F894204A7980F812
:1057400095208A7980F89620C97980F897105F496A
:1057500008310A7880F898204A7880F899208A7869
:1057600080F89A20CA7880F89B200A7980F89C20DB
:105770004A7980F89D208A7980F89E20C97980F83E
:105780009F10524918310A7880F8A0204A7880F892
:10579000A1208A7880F8A220CA7880F8A3200A790C
:1057A00080F8A4204A79C2F3400363F35F0280F8D3
:1057B000A5208A7980F8A620C97980F8A7104349E6
:1057C00020310A7802F0010280F8A8204A7880F897
:1057D000A9208A7880F8AA20CA7880F8AB200A79B4
:1057E00080F8AC204A7980F8AD208A7980F8AE2024
:1057F000C97980F8AF10354928310A7880F8B0208F
:105800004A7880F8B1208A7802F0030280F8B2204A
:10581000CA7880F8B3200A7980F8B4204A7980F8F1
:10582000B5208A7980F8B620C97980F8B710274961
:1058300030310A7880F8B8204A7880F8B9208A7820
:1058400080F8BA20CA7880F8BB200A7980F8BC209A
:105850004A7980F8BD208A7980F8BE20C97980F81D
:10586000BF101A4938310A7880F8C0204A7880F889
:10587000C1208A7880F8C220CA7880F8C3200A79CB
:1058800080F8C4204A7980F8C5208A7980F8C6203B
:10589000C97980F8C7100D4940310A7880F8C820CE
:1058A0004A7880F8C9208A7880F8CA20CA7880F8B7
:1058B000CB200A7980F8CC204A7980F8CD208A79EB
:1058C00080F8CE20C97980F8CF1010BDEF070020F6
:1058D0007CB50121082000F0ABFD4FF40050ADF87D
:1058E000040010248DF8074001208DF8060001A95E
:1058F0001548FDF759FF0121092000F099FD01210C
:105900001248FDF7A3FF0820ADF8000004208DF831
:1059100003000F4E03258DF8025069463046FDF70F
:1059200043FF08213046FDF7C4FFADF800408DF875
:1059300003408DF8025069463046FDF735FF1021CF
:105940003046FDF7B6FF7CBD001401400002300078
:10595000000C0140FEE7000038B50121082000F0EE
:1059600067FD4FF44060ADF8000048208DF803005B
:1059700003201E4D8DF8020069462846FDF714FFEE
:1059800029152846FDF78EFF194CE914E070A07028
:105990002846FDF787FF60712071FDF7ABFFA082FD
:1059A000E0820020A071E07120726072A072114844
:1059B00090F84A10104849B101290BD002290FD0A4
:1059C00003290CD1C17841F0030107E0C17821F02F
:1059D000030103E0C17821F00301491CC17038BD07
:1059E000C17821F00301891CF8E70000000C014098
:1059F000B0080020C0020020AF0700202DE9F05FB2
:105A00008B4D4FF480612846FDF74CFF0446E914A6
:105A10002846FDF747FFDFF81C920646002599F857
:105A20000200A8462F46844205D089F80240FDF7BF
:105A300061FFA9F8140099F8030084420AD0B9F86C
:105A40001400FDF73FFF1E2804D389F803405CB320
:105A50004FF0010899F804004C46864203D02671A5
:105A6000FDF748FFE0826079864207D0E08AFDF7C3
:105A700029FF1E2802D36671C6B10027E1786E485F
:105A80000029017914D021F0020101716279A24646
:105A90008AB121F001010171807841067ED4674A04
:105AA0001178CB070AD00FE00125D3E70127E5E7FE
:105AB00041F00201E9E741F00101ECE70DB1002FEF
:105AC0006CD155EA070369D05D4BDB7803F0030422
:105AD000032C00D903249146C9074FF0010B4FF066
:105AE00000061AD03DB1FDF705FFAAF80C00AAF890
:105AF00010008AF800603FB1FDF7FCFEAAF80E0026
:105B0000AAF812008AF8016055469AF803004FF48B
:105B1000FA7A4FF47A77A8B12AE01DB1032C01D2AA
:105B2000641C6BE0DFB3D4B3012C02D0641EE4B27A
:105B300064E04449496CB1F5FA6F5FD2C0065DD5A7
:105B400000245BE0687958B3A889FDF7BBFE504597
:105B50000ED385F800B0288AFDF7B4FEB84207D30B
:105B6000B9F81010C831A9F81010FDF7C3FE28824B
:105B70006879A8B9E87898B1E889FDF7A3FE50459F
:105B800017D385F801B0688AFDF79CFEB84210D3A0
:105B9000B9F91010C82907D3C83902E03EE02DE05A
:105BA00007E0A9F8101001E0A9F81060FDF7A2FEC7
:105BB0006882B8F1000F07D0287828B9B9F810101A
:105BC00001F57A71A9F81010687988B1687878B908
:105BD000E88AFDF777FE1E280AD1B9F91010B942FC
:105BE00004D3A1F57A71A9F8101001E0A9F81060AA
:105BF000E87800B12E70687900B16E701048C178F5
:105C000064F30101C170104854B1012C0BD0022C77
:105C10000CD0032C02D1032180F84A10BDE8F09F7C
:105C200080F84A60FAE780F84AB0F7E70221F3E724
:105C3000000C0140B0080020BF070020F80A002037
:105C4000AF07002050010020C0020020704700F084
:105C50001F02012191404009800000F1E020C0F8BE
:105C60008011704700F01F0201219140400980001F
:105C700000F1E020C0F88011704700F01F02012100
:105C800091404009800000F1E020C0F80011704709
:105C900000F01F02012191404009800000F1E02046
:105CA000C0F800117047000070B50F23C478017868
:105CB0000122F4B1144C2468457804F4E064C4F57E
:105CC000E064240AC4F10406E3408478B5401C4033
:105CD0002C4301F1E021230181F80034007800F029
:105CE0001F018A404009800000F1E020C0F8002137
:105CF00070BD01F01F0082404809800000F1E020E3
:105D0000C0F8802170BD00000CED00E0024908439E
:105D100002490860704700000000FA050CED00E041
:105D2000024A1140014302480160704780FFFF1F93
:105D300008ED00E0F0B5254843F69821B0F90400DD
:105D4000884201DB012200E000222148817841F0F5
:105D5000800383701D481C064FF00001A0F108006D
:105D600011D5DB070FD01B4BDB791C060BD51A4C6A
:105D700094F84A40032C06D103F07F03322B02D95A
:105D8000037813B1FAB9017018E08578134B43F624
:105D9000095435B11D888688AD1BADB2A54200D926
:105DA000817082B1457875B98678012546B11E8823
:105DB0008788F61BB6B2A64203D80570817002E050
:105DC0008570198881804270F0BD000010060020A7
:105DD000AF070020DF070020C00200207807002066
:105DE00010B54FF440514FF00060FFF799FF62B6D5
:105DF00010BD00002DE9F05FDFF8F0910026B9F842
:105E0000202040F272637A497A4835469A4208D98E
:105E10008278521CD2B28270022A04D301200881F7
:105E200001E085700D811D20FFF711FF714CDFF837
:105E3000C8E1C034A4F1B800A77E90F83810DFF8AC
:105E4000BCB18F427ED0E776A176626A036B5A437B
:105E50004FEA124A99F80820120702D51EF80120CD
:105E600000E00A4694F812C0BCF1010F09D004EB1F
:105E70004206B6F902C0C4F828C0B6F90460E6626A
:105E80000CE043F6FF7CC4E90A5C90F83DC05FEA91
:105E9000CC7C01D012B102E0052A00D1012600EB32
:105EA00047074FF0804CBF893F04B7FBF3F3E36132
:105EB000476BBCFBF7F7276294F813C0BCF1000FE7
:105EC00006D0BCF1010F05D03B4403EBD3735B104C
:105ED000636201E03B466762DFF824C14FF6FF775B
:105EE00007EA8307ACF808709BF8007090F80A8006
:105EF00090F83DC0082F08F003070CF0030C05D004
:105F000067450BD1B8F1000F05D008E0674505D013
:105F1000B8F1000F03D05B42636200E06562C6B176
:105F2000636A002B03D006DD228D05E00AE0354BC5
:105F300033F8122000E0A28DA4F86020227822F02D
:105F4000200222709BF80020042A07D0082A05D0DE
:105F500019E0B4F8603003EB0A02EDE780F8405036
:105F6000656299F80800000707D51EF80100264968
:105F700001EB400030F8020C03E0224800EB410046
:105F80004088A4F860002149606A09883E3148438E
:105F9000B4F8601001EB204006B21D20FFF76DFE43
:105FA000606A002807D021784FEA81600ADD002866
:105FB00004DAA08D09E0B4F8600006E0E06AB042BF
:105FC00008DB0CE0002802DA208D208208E0A06ABD
:105FD000B04204DD208241F02000207000E02682E3
:105FE000257565752586BDE8F09F0000C00200207C
:105FF000480C0020480100207CC600086F070020E4
:10600000DC0B00208EC60008A8C60008240400404F
:1060100043184FF48042934210DD904202DD104657
:1060200000210BE0914202DD0020114606E08003D2
:10603000B0FBF3F000B2C0F5804109B241EA004084
:106040007047F0B541F2F1130022C3600E24826262
:1060500004824BF2660508264561068343F6FF7706
:106060004283878340F2492E4FEA873CC0F808E01C
:10607000C0E9082CCB608A620C824D610E834A8392
:106080008F83B4208860C1E9082CF0BD00218162B3
:106090000949C1600E21018208494161082101833B
:1060A0004FF44041418343F6FF7181830907016248
:1060B0000349416270470000B6A001001C0C0100BA
:1060C00000C0FF0F064941F681600880054801685D
:1060D000054A01F4E06111430160BFF34F8FFEE711
:1060E000442C01400CED00E00400FA05F8B5012154
:1060F0000D2000F09DF94FF4E060ADF80000182489
:106100001D4E8DF8034003258DF802506946304638
:10611000FDF74AFBB1153046FDF7CBFB7115304654
:10612000FDF7C7FB31153046FDF7C3FB4FF4604068
:10613000ADF800008DF80340104C8DF80250694610
:106140002046FDF731FB61142046FDF7B4FB4FF408
:1061500080412046FDF7AFFB4FF400412046FDF79C
:10616000AAFBA014ADF8000048208DF80300694692
:106170002046FDF719FBF8BD00080140000C014066
:106180002DE9F0410121CE028CB0304600F050F9EB
:10619000DFF87081404601F0BDFC08A801F0E6FE82
:1061A0004FF45860ADF824000024ADF820402020C2
:1061B000ADF822000125ADF826408DF8285008A939
:1061C000404601F085FE0021404601F0D8FE4FF622
:1061D000FF71404601F0DDFE01220021404601F042
:1061E00069FE0121404601F051FC04A801F069FC60
:1061F000ADF81060A802ADF81200ADF8144081208F
:10620000ADF816002803ADF81800ADF81A40ADF847
:106210001C4004A9404601F043FCADF808400820AA
:10622000ADF80A006027ADF80C408001ADF80070B1
:10623000ADF80440ADF80E00ADF80240ADF80640F0
:106240006946404601F026FD6946404601F068FD7A
:106250006946404601F0AEFDADF8045040F61450DA
:10626000ADF80070ADF80600ADF80840ADF80C4090
:10627000ADF80250ADF80A40ADF80E406946404610
:1062800001F0DCFD0121404601F024FC08214046DC
:1062900001F040FD3146404601F082FD08214046B4
:1062A00001F0C6FD3146404601F0FAFD702140463E
:1062B00001F003FE18208DF82C008DF82D408DF88C
:1062C0002E408DF82F500BA8FFF7EEFC0D480C3038
:1062D000018841F0800101800A481430018841F0B2
:1062E00001010180001F04800121404601F0FCFBF8
:1062F0008DF828500121404601F000FC0CB0BDE8AB
:10630000F0810000002C0140704740F213414160D1
:10631000082181608621C1604FF4804101614942BA
:10632000416100210162C162704701627047000053
:1063300010B501884288891A09B20183B1F5005F5E
:1063400002DBA1F5804104E011F5005F02DC01F5FC
:1063500080410183B0F9182041685143C1618368CD
:10636000846A5343C2681B12624303EB2222036A0E
:106370001A44114402628A13426241698A4203DB71
:1063800001698A4200DC11468A1AC0E90A21028E9C
:106390004FF40373594302EBA13202860B4A127881
:1063A000082A04D10A4A936F03EBA1319167B0F92F
:1063B0003010B1F5804F02DDA1F5804103E00029E6
:1063C00002DA01F58041018610BD00006F07002050
:1063D000600C0020034A516821F4404101435160A0
:1063E0007047000000100240044A0029516901D0A2
:1063F000014300E0814351617047000000100240FA
:10640000044A0029D16901D0014300E08143D161F0
:106410007047000000100240044A0029116901D0B1
:10642000014300E081431161704700000010024009
:10643000044A0029916901D0014300E08143916140
:106440007047000000100240044A0029D16801D0C2
:10645000014300E08143D16070470000001002401A
:106460002DE9F041274C4FF4807631462046FDF768
:1064700019FA850080212046FDF714FA45EA400507
:1064800040212046FDF70EFA0543EDB23146204685
:10649000FDF708FA870080212046FDF703FA47EA56
:1064A000400740212046FDF7FDF90743F8B2A84216
:1064B000DBD131462046FDF7F5F9870080212046E3
:1064C000FDF7F0F947EA400740212046FDF7EAF9D9
:1064D0000743F8B2A842C8D131462046FDF7E2F999
:1064E000870080212046FDF7DDF947EA400740217B
:1064F0002046FDF7D7F90743F8B2A842B5D12846A0
:10650000BDE8F0810010014010B50268416802FB4F
:1065100002F301FB0133B3F1805F11D91B0E103B75
:106520000A4C9BB212B234F8133009B25A435943A1
:1065300042F38F3241F38F31C0E90221012102E0A1
:10654000C0E902210021017410BD000068BC0008F0
:106550002DE9F05FF848F94902880B889A1A92B23F
:106560000F2A70D309880180F5480024827852B13F
:10657000818AB1F5967F02D2491C818204E084822F
:10658000521E827000E084828146C078401E01283D
:106590000ED8B9F8161047F230524846914203D24D
:1065A000491CA9F8161005E0C48289F8034001E0EF
:1065B000A9F81640E3480246C189D2884B0703D4A4
:1065C0008B0701D4CB0702D042F4007201E022F421
:1065D0000072C2808346080702D45846C90604D513
:1065E000BBF8061041F0010102E0C18821F0010171
:1065F000ABF80610D348FCF7DFFED348B0F93A00F9
:10660000B0F5804F02DAD049401C02E0CE494FF489
:106610008040DFF838A34887C94DDAF8500041F6CA
:10662000CC413835884203DDA86820F01000A8600E
:10663000C749DFF82083C84E088828B1401E08806B
:10664000EC73347045E062E199F8020008B1032868
:1066500005D9C248017821F00201017039E0B5F88E
:10666000420088B1BBF806005F4641041FD4F98997
:10667000CA061CD409071AD4810618D4000516D4FA
:10668000FDF7C4FB98B904E0B54949F6816008807C
:106690002CE0F88841070AD4C10508D4010706D4C4
:1066A000810404D4C00602D4B87BC00711D0EC73B7
:1066B0003470FDF7ABFB30B1404600F85E4F4480CC
:1066C000447688F87640A748A749C4830C8080F8B0
:1066D0002840B5F8420048B1401EA5F842009F4846
:1066E000017821F002010170EC730BE09B48017806
:1066F00041F0020101703078012804D19B480078F4
:10670000062800D134703078DFF864E201270A28C7
:1067100071D2DFE800F0FDFC05FCFBFAFC70F9F833
:1067200002F0FAFAB9F82210491C8AB2A9F822201C
:10673000DAF8440040F62821884202DAA9F822401B
:1067400016E0814840F6CC41C068884210DB83489F
:1067500043F69911B0F90400884209DBB2F5FA7FDB
:1067600006D398F800201AB9A9F8224088F80070DA
:106770008048008868B199F80610491CC9B289F8A8
:106780000610022905D37C4889F806400188491C77
:1067900001809BF8060040F2DC5B000614D585F80A
:1067A000EE40C5F8DC405123B5F934101A460020FC
:1067B00000F090FCA8866448C068B0F5F67F03DA64
:1067C000AC86EC73347004E0E87B092814D002280E
:1067D0006FD0A5F83441B5F84400E8B1A9F82240DB
:1067E000DAF8442041F288318A4229DA98F8002008
:1067F000012A1FD024E034E24F484430FDF7B4F9B9
:10680000FCF750FEDAF84410C9F8341041F27C511C
:106810000920C9F8241033E3B8F81410A986D8F871
:106820002C10C8F83410D8F82810C8F83010A5F883
:10683000447059E0504988F800400C804D490C8064
:106840004649B1F90410B1F5A47F15DBB5F9341050
:10685000002911DAC5F8DC4085F8EE4040F2333209
:1068600013460020C9F82C4000F034FCA88610F133
:10687000A30F39DBAC8637E095F84A10022908D01F
:106880003E49C978B7EB511F14D095F82C0148B197
:1068900002E095F82C0110B1C5F8DC4006E06FF07D
:1068A000F40001E06FF40560C5F8DC0085F8EE70D7
:1068B00006E095E0C5F8DC4085F8EE40C9F82C40CC
:1068C0002E48B5F93410C078B7EB501F05D0B5F895
:1068D000DC00642300B25A4603E04FF47A735A0096
:1068E000002000F0F7FBA88698F85E00244A414695
:1068F00042F6E063042818D020484FF49A7CC07810
:10690000B7EB501F05E01BE1F6E061E15CE10AE056
:1069100063E1DAF844004CD0B0F5FA7F03DAB8F955
:106920000A00604540DDBDE8F09F1648806D0028F4
:106930002ADB074629E00000100B00207807002022
:1069400088020020480C002058050020500100203B
:106950007C070020600000206F0700201006002048
:10696000442C0140780A0020140000207007002009
:10697000700200201A0000201C000020D707002011
:10698000840B0020940900204742C82F04DAB1F993
:106990001470B7F5F77F07DB9842C4DDB8F914002F
:1069A000C730B0F5C77FBED8347085F8EE40548349
:1069B000B9E7584503DAB8F90A106145F4DDB5F8CE
:1069C000441040F6C417491C89B2A5F84410B942D6
:1069D000EAD2FB49C9680029A5DC9842E4DAA2E7BB
:1069E000B5F8340140F6B831884206D2F54A12783B
:1069F000D20702D1401CA5F8340182B25A4502D810
:106A000042F6CC4103E0A5F8341143F26661C8F8C0
:106A10007C10DAF84400C9F8340089F80B70EA4FAA
:106A2000A5F8444085F8EE40787F4E46E0B1F87F07
:106A3000B8B3A88DB5F9341000B20A23052200F0CE
:106A400049FBA886FC777C77B5F91A01B5F91811CE
:106A500088423EDAF17901F1010111F0FF01F17193
:106A60003ED0F471401C36E04FF48040A5F8E800B9
:106A7000E96A814200DA0846D44900B2308491F8CC
:106A80004D1049B995F84A1031B12A89C2F3C003B3
:106A9000C2F30022934205D13623B5F93410052202
:106AA0000AE013E0012903D0022901D0032906D00E
:106AB000B5F93410DA23242200F00CFB07E0B5F915
:106AC000341040F2991340F26662F5E7A320A886DD
:106AD000BAE703DD801EA5F81A0101E0A5F81A1136
:106AE000B5F934104FF48040814201DDA8861AE7E1
:106AF0000029FCDAAC8616E7D5F8E0004EF66021F6
:106B0000884202D2401CC5F8E000E87B082803D187
:106B1000D5F8E00088420FD33470A86820F40060F4
:106B2000A860C10502D520F0080001E040F008008F
:106B3000C5F8E040A860F6E6BDE8F05F03F088B86D
:106B4000E87B092813D003282DD0B5F934104FF471
:106B5000237702282BD0CC231A46002000F0BAFA63
:106B6000A88600F5A370B842C1D8AC868AE1D9F8EE
:106B700028004E46401CC9F82800022809DDB08EC6
:106B8000012301B2B08C052200B200F0A3FAB46276
:106B900070638C48B18E5C300180BAF8441041803B
:106BA000FCF7FAFFA2E789F80C70032068E140F2D5
:106BB00047121346002000F08DFAA88600F5A37056
:106BC000B84294D8AC865AE1BDE8F05F04F0E2BE6A
:106BD0009EF8000009287DD0A5E685F8114195F8BA
:106BE0002C0180B1C5F8DC40DAF85000784A40F357
:106BF00011008303C8F82C00801093628103C8F849
:106C0000280074488162A9F82240DAF8441041F261
:106C10008830814209DA98F80010012905D16E48C0
:106C200088F8004004806D4804806D496D4B0888E9
:106C3000401C82B26C480A80C82A04D390F800C075
:106C4000BCF1010F19D0B2F57A7F04D390F800C0DF
:106C5000BCF1020F11D0B2F5FA6F02D30278032A09
:106C60000BD0E87B801E08286FD2DFE800F010C749
:106C7000FDFC056E8204BFE555E604700C80BBF890
:106C8000061021F40061ABF806101F70E9E7DAF88E
:106C90004400822805DA55480178062901D004709D
:106CA0000AE1FCF757FE9AF80000400615D5504857
:106CB0008078042811D0DAF84410504682290CDA82
:106CC000817A9AF83D0001F0030100F0030081424F
:106CD00003D000E0D6E001F0ABFE3078B3460628E2
:106CE000CAD08AF83F40DAF85000394A40F3110020
:106CF0008303C8F82C00801093628103C8F8280031
:106D0000344856468162FCF7CDFB89F80B70B5F824
:106D10001801A5F81A01706CA5F88640B0F5437FFC
:106D200014DD4FF48040A5F88400A86840F480602A
:106D3000A86096F8381005299ED100BF40F01000D9
:106D4000A86002208BF80000EDE5BCE04FF4804124
:106D5000A5F88410A96821F48061A96040F28A2115
:106D6000884204DA3078400601D402F047FEA86871
:106D7000E4E7DAF84400B0F5437F03DA1B48017812
:106D800006298CD11B48017821F040010170FCF7E5
:106D900089FB43F6FE70A5F81A01E035FCF7DAFD31
:106DA000154810F8341F21F00101017009492C60C9
:106DB0008C6207498C62082131704464B3E500009D
:106DC00058050020F80A00206C0E0020A40E0020B8
:106DD000480A0020180A00201C0000201A00002089
:106DE000240100202201002026010020700700203D
:106DF000740400207E070020600C00209BF8060031
:106E0000C006A1D43348407810F00C0F9CD0DAF8BB
:106E100044005746B0F57A7F34DDFCF79BFD3878A7
:106E2000400611D52C48807804280DD0786C822833
:106E30000ADAB87A97F83D1000F0030001F0030178
:106E4000884201D001F0F4FD87F83F40B7F85000C8
:106E5000A88601B24FF48040814200DDA886FCF78D
:106E600021FBA86801E023E00EE040F48060A86008
:106E700097F838100529A1D140F01000A860022031
:106E8000307050E534704EE5DAF84400B0F5437FD9
:106E900004DA1248017806297FF401AFBBF8061026
:106EA00021F02001ABF80610FCF754FD0420E7E7C1
:106EB0000A480078062801D0377034E509208EF89A
:106EC00000000520DCE7044884700448047088F85A
:106ED0005E400FE6D70700207404002070070020F2
:106EE00030B585B001210420FFF7A2FA4FF400402D
:106EF000ADF8100048208DF8130004A91848FCF7DD
:106F000053FC01210846FFF77BFA40F68C20ADF8D0
:106F1000040003240020ADF80040ADF80200ADF8F5
:106F200006004FF080456946284600F0D1FF1C203E
:106F30008DF80C008DF80D408DF80E4001208DF875
:106F40000F0003A8FEF7B0FE01221146284600F00C
:106F500099FE0121284600F0C7FD05B030BD0000B4
:106F600000080140704700002DE9F041304CE07806
:106F700000285AD12078002857D0401E10F0FF007A
:106F8000207052D14FF49670208272B6294F45F28C
:106F9000AA50A7F872000020FCF762FA264D1320D1
:106FA0002860FCF76FFAA8BB3420E8600220286153
:106FB000224E6E61286940F040002861FCF762FAB9
:106FC00040BB00211E4A08465FEA255312F800C064
:106FD000BCF1FF0F00D00121401C80B29842F5D3D4
:106FE000C1B9C4E9067639260127A06910F8011B4A
:106FF00010F8012BA061E06901EB022102886A61AF
:107000002F6120F8021BE061FCF73CFA10B9761EF4
:10701000B6B2EAD20120FCF723FA62B601F05CFDB9
:107020000848816821F480418160BDE8F08100005A
:107030006C070020A40E00200020024000FC000885
:1070400000FC0008C00200201948016841F010014E
:107050000160016821F003010160016841F0020153
:10706000016014484168416041684160416841F4F1
:1070700080614160416821F47C11416041680E4AA1
:1070800011434160016841F080710160016889012C
:10709000FCD5416821F003014160416841F00201E3
:1070A00041604168C1F381010229FAD170470000B3
:1070B00000200240001002400000280830B5044CB7
:1070C000039D6080A180E2802381658130BD000046
:1070D0003C0C00200A44824201DA10B27047C91AFF
:1070E0008142FBDD08B270472DE9F04F4748DFF8D9
:1070F00020A1DFF820B1C17F477A0468464800220A
:10710000DFF82091466C45484FF0010E80298578C4
:107110004348836834D301F01F0C5AF82C100C42FA
:107120000146096802D041F4805101E021F4805108
:1071300001605FEAC14C1ED45FEA814C1BD599F80F
:107140000CC0C8465FEACC7C0BD05FEAC31C12D4EB
:10715000A8F80C209BF8008028F002088BF800802B
:1071600009E0322E07DC5FEA857C04D55FEA035C28
:1071700001D4A8F80CE04FEA113C6CF34D310160EA
:10718000802F24D307F01F075AF827100C420168FC
:1071900002D041F0040101E021F0040101604C073C
:1071A00011D44C050FD599F80C70FF070BD0DF01F7
:1071B00009D4A9F80C209BF8007027F002078BF87F
:1071C0000070C0F89C208C0864F38A21016099F853
:1071D0000C40E40714D1322E10DC046866070DD58C
:1071E0001B050BD4E30409D5AB0707D5D0F89C30B9
:1071F0004EF66024A34205D9A9F80CE0C0F89C2003
:10720000BDE8F08F5B1CC0F89C30F9E71806002041
:10721000B8C100081006002050010020BF07002060
:10722000C0020020480C002010B5F9F7F1FD0F480E
:10723000018821F0020101800C49183109880C4AAB
:10724000928E1144094A3432118008490C390A8857
:1072500042F001020A80011D0A884FF6ED531A40E0
:107260000A80018841F01201018010BD0C04004029
:1072700074040020130A03700A70704705484FF623
:10728000FF620188491C89B20180914201D300212B
:1072900001807047C80800200F4810B5016841F010
:1072A0000101016041680D4A1140416001680C4ACA
:1072B00011400160016821F480210160416821F4DE
:1072C000FE0141604FF41F018160FFF7BDFE0549DB
:1072D0004FF00060086010BD001002400000FFF891
:1072E000FFFFF6FE08ED00E04FF0E02005494161A8
:1072F000054AF02182F8141D0021816107210161F6
:1073000070470000DFA501000FE000E02DE9F04725
:10731000DFF8B090B9F800004FF0000400064DD53A
:10732000294D6888401C6880FBF74AF9274E284B96
:10733000284832786A7093F80080072726494FF072
:10734000C80CB8F1010F03D0244AD288E2B12EE074
:1073500072B1012A12D0C28842F40062C2808868E9
:1073600040F00400886003202870052030701BE086
:10737000C28942F00802C2810120F5E7C28942F0C9
:107380001002C2810220EFE7154A15786D1CEDB29C
:107390001570032D08D91470C28842F40062C280AF
:1073A000886840F0040088601F70A1F842C0002087
:1073B0004FF49661401C80B28842FBD3A9F800408C
:1073C000BDE8F087102C01405C070020700700200A
:1073D0006F070020480C0020C0020020100B002086
:1073E0008A020020704700002DE9F0434FF08040F2
:1073F000018A21F001010182AA48007800287CD18D
:10740000A94FF87B002878D1A848406C322874DC5A
:10741000A7488068DFF89C924104A74DB9F80400A2
:107420004FF0000403D4401CA9F8040024E1002814
:1074300074D02978012611B1012912D013E14946EF
:10744000B0F5BE7FFAD92E70CC718C71EC702C72B5
:10745000287A0A18401CC0B2147228720F28F7D379
:1074600001E1B9F802204946824201D9EE7100E0FB
:10747000EC7190488A7908300F2A15D2CB79082B05
:107480000BD2C3F10708EB7912F800C003FA08F336
:1074900063441354CA79521CCA71CA79082A03D1A9
:1074A0008A79521C8A71CC7199F80610C8460F2946
:1074B00073D10D21FAF71CFEA881010A6970C0B2D0
:1074C000A87088F8064098F816208A4265D198F886
:1074D0001510814261D198F80BC07849032302222C
:1074E0007748BCF1000F10D0BCF1010F02D0BCF105
:1074F000020F14D080F86A2000E0C7E091F800C0C5
:107500002CF00C0C0CF1080C0FE080F86A6091F87C
:1075100000C02CF00C0C0CF1040C06E0A5E080F887
:107520006A3091F800C04CF00C0C81F800C098F85B
:107530000C10B6EB111F04D180F86E4087F84A405A
:107540000EE0B2EB111F04D180F86E6087F84A603C
:1075500006E0B3EB111F03D180F86E2087F84A20B4
:107560000B0717D001F00F01012901D0022915D016
:1075700080F86C602C7198F80D102A7906FA02F3E5
:107580000B406B71082A41D2DFE802F00B0F401666
:10759000212C333A80F86C40ECE764E080F86C20F2
:1075A000E8E713B380F8704030E013B180F8506022
:1075B0002CE080F8504029E023B180F8656087F81E
:1075C000076123E080F8654087F807411EE023B19A
:1075D00087F8F94080F84D4018E087F8F96080F8A6
:1075E0004D6013E013B180F868600FE080F86840E8
:1075F0000CE013B180F8666008E080F8664005E0B2
:1076000013B180F8676001E080F86740521CD2B285
:107610002A71082AB1D398F80E108A0704D587F882
:10762000F56080F8646005E0264A87F8F54080F848
:1076300064409481C90702D080F8294001E080F8B5
:10764000296098F8111000F86D1FC2781E48012AB1
:107650001ED001B3012921D04FF48051A0F876103B
:107660001A493C200870A9F80240A9F80440B9F86A
:107670000210491CA9F80210B9F80210B1F5FA7FFE
:1076800004D940F2F511A9F802102C70BDE8F0837E
:1076900044F21C71E2E74FF40051DFE741F255512B
:1076A000DCE700006F070020C0020020500100202E
:1076B000001001408C0E0020F8060020EC04002091
:1076C000A40E0020480C0020580500206C07002064
:1076D0002DE9F05FFCF73EF98B4D2888A5F10406F3
:1076E000C0070DD0308820F008003080288820F0B6
:1076F0000900288002F082F9BDE8F05FFCF7C6BD02
:107700002888DFF80892DFF80882824C80071AD5B3
:10771000B9F8001041F00101A9F80010B8F8000014
:107720007B4914315030088028884FF6F9510840C1
:107730002880308840F004003080FEF791FE84F805
:107740003C00BDE8F09F2888734F4007288872D519
:1077500020F004002880FEF783FE94F83C1081425C
:10776000EFD1308820F004003080FCF78DFD2078C8
:10777000410605D594F8541094F83B209142E0D08E
:107780003978400621F00201397004D5FDF79AFCE2
:1077900097F82F7004E094F83C00FCF72DF90746A9
:1077A000DFF86CB140F68C2A0BF1180B062F48D28B
:1077B00094F83800B8423FD03846FCF7A1F820785A
:1077C000C00716D094F83A0094F8391000F003027C
:1077D000914206D0A17A00F0010001F00101884237
:1077E00015D1FCF77DFAF9F75FFBFCF773FD38461E
:1077F00081E0FCF775FAF9F757FBFCF76BFD3846AB
:10780000FCF78EFA207840F00100207099E7288874
:1078100020F008002880206B810801EBD000504543
:1078200016D200BFB8F800100844ABF8000030884A
:1078300040F0080003E00DE0308820F008003080C0
:107840007FE7B9F8001041F00101A9F80010DEE768
:107850005046E7E70007288828D520F00800288050
:10786000308820F008003080FEF7FAFD84F83C00F4
:10787000FCF70AFD387820F00200387020784006C6
:1078800004D5FDF71FFC97F82F5004E094F83C0056
:10789000FCF7B2F80546062DB8D294F83800A84295
:1078A000B4D0FCF71DFAF9F7FFFA21E0C0062888EA
:1078B00025D520F010002880308820F0100030807E
:1078C00097F838000C2802D2401C87F83800387826
:1078D00040F002003870FDF7F5FB97F82F507878EC
:1078E00084F8390094F83800A8428FD0FCF7F8F9F2
:1078F000FCF7F0FC2846BDE8F05FFCF711BA4EF249
:10790000BE11084028801CE710040040000400401D
:107910002404004050010020740400202DE9F04FA1
:10792000514F85B0388820F0010038804E4800263D
:10793000103006804D4CDFF838A14FF0010894F864
:107940005C0042F63029C10774D072B6494881699B
:1079500041F400718161816941F4806181614FF47A
:107960000040FEF737FD444D00212846F8F7DCFFC4
:1079700000212846F8F7CEFFDFF800B10021584675
:10798000F8F7C8FF00213E48FBF7E6F82846F9F76C
:10799000EDF85846F9F7EAF84FF46020CDE9020611
:1079A0008DF8056000968DF810808DF8048069468A
:1079B0002846F9F76DF901231A460F212846F9F7F1
:1079C000B8F901212846F8F7A5FF00204946401CD8
:1079D00080B28842FBD328462E600121F9F7E8F9EE
:1079E00028688007FCD524484C30006894F85C1067
:1079F00021F001012144A1F85000F8F79FFF62B681
:107A0000FDF76EFA47F69061AAF8001094F85C0052
:107A1000401CC0B284F85C000C2822D212491431F8
:107A2000A1F80080388840F00100388005B0BDE83A
:107A3000F08FFFE7134920F00100085A124908802F
:107A4000114945F65800083908800F4846F6580194
:107A5000001F01800C4920200C390880AAF80090F2
:107A6000D4E70320A070E1E7000800407404002080
:107A70002C08004000100240002401400028014072
:107A80000800024074BD0008202C01400029018834
:107A900002D041F0800101E021F0800101807047B7
:107AA00010B50A884B88CC881A438B8823431A4325
:107AB0000B891A434B8989891A430A43A0F8442049
:107AC00010BD0021018041808180C1800181418100
:107AD000818170470029818802D041F0010101E0D5
:107AE00021F00101818070470029018802D041F016
:107AF000010101E021F0010101807047002930F807
:107B0000441F02D041F4004101E0C1F30E010180A5
:107B1000704700004B4910B5884202D10121C414BE
:107B200086E0B0F1804F09D0474988420DD101214C
:107B30000220FEF771FC0021022064E001210846CA
:107B4000FEF76AFC002101205DE04049884206D131
:107B500001210420FEF760FC0021042053E03C4991
:107B6000884206D101210820FEF756FC002108209A
:107B700049E03849884206D101211020FEF74CFC2B
:107B8000002110203FE03449884206D10121202005
:107B9000FEF742FC0021202035E03049884202D126
:107BA0000121441444E02E49884202D10121CC0431
:107BB0003EE02C49884202D101210C0538E02A49D7
:107BC000884202D101214C0532E02849884206D181
:107BD00001214020FEF720FC0021402013E0244931
:107BE000884206D101218020FEF716FC002180206A
:107BF00009E0204988420AD1841501212046FEF778
:107C00000BFC00212046BDE81040FEF705BC1A49D8
:107C1000884202D101210C040AE01849884202D1AD
:107C200001214C0404E0164988420AD101218C0448
:107C30002046FEF709FC2046BDE810400021FEF773
:107C400003BC10BD002C01400004004000080040AF
:107C5000000C0040001000400014004000340140BF
:107C6000004C014000500140005401400018004009
:107C7000001C004000200040004001400044014042
:107C800000480140002A828901D00A4300E08A436B
:107C90008281704730B5028C22F001020284028C8E
:107CA0008388048B22F0020224F073050C882C4395
:107CB0000D8915434A882A43114DA8420BD0114D16
:107CC000A84208D0104DA84205D0104DA84202D0BD
:107CD0000F4DA8420DD122F008054A8923F44073C4
:107CE0002A4322F004058A882A438D891D43CB89C3
:107CF0002B4383800483C9888186028430BD0000C1
:107D0000002C01400034014000400140004401408B
:107D100000480140028B22F008020A4302837047A8
:107D200070B5028C22F010020284028C8488038BCE
:107D30000D8823F4E6464FF6FF7303EA0525354325
:107D40000E8922F0200203EA061616434A8803EA47
:107D500002123243104EB04202D0104EB04215D142
:107D600022F080064A8924F4406403EA0212324376
:107D700022F040068A8803EA021232438E8903EA1F
:107D800086062643CC8903EA840434438480058331
:107D9000C9880187028470BD002C01400034014075
:107DA000028B4FF6FF7322F4006203EA01211143B4
:107DB0000183704770B5028C22F480720284028CB9
:107DC0008488838B0D8823F073031D4322F4007392
:107DD0000E894FF6FF7202EA06261E434B8802EA1E
:107DE00003233343104EB04202D0104EB04215D19F
:107DF00023F400664B8924F4405402EA03233343FE
:107E000023F480668B8802EA032333438E8902EAD7
:107E100006162643CC8902EA041434438480858301
:107E2000C9888187038470BD002C01400034014063
:107E3000828B22F008020A438283704770B5028C5D
:107E400022F480520284048C8288838B0D8823F470
:107E5000E6464FF6FF7303EA0525354324F4005642
:107E60000C8903EA043434434E8803EA0636264379
:107E7000094CA04202D0094CA04205D122F4804412
:107E80008A8903EA8212224382808583C988A0F806
:107E90004010068470BD0000002C014000340140F9
:107EA000828B4FF6FF7322F4006203EA0121114333
:107EB00081837047018582827047828822F0700238
:107EC000828082880A4382807047A0F84010704701
:107ED00030B502881B4B1C4C98420DD0A0420BD0F1
:107EE000B0F1804F08D0194DA84205D0184DA842D6
:107EF00002D0184DA84203D122F070054A882A43C7
:107F0000154DA84206D0154DA84203D022F4407565
:107F1000CA882A4302808A8882850A880285984214
:107F20000AD0A04208D00E4A904205D00D4A904295
:107F300002D00D4A904201D1097A01860121818245
:107F400030BD0000002C014000340140000400401E
:107F500000080040000C00400010004000140040E9
:107F60000040014000440140004801404FF6FF71CD
:107F7000818000210180C180418001727047002909
:107F8000018802D041F0020101E021F002010180EC
:107F900070470029018802D041F0040101E021F07E
:107FA0000401018070470000194810B54079002392
:107FB00000F003011748022927D0174A01881488C6
:107FC000611A89B201240F290BD3118801808168BD
:107FD000002900DA4942052903DD10490978022900
:107FE00005D0417F012906D01188418010BD44771A
:107FF000C3771188418041881288511A89B240F2B2
:108000001A629142F2D3C47710BD437710BD0000CD
:10801000D70700206C0E0020780700206F07002093
:1080200080092830FF2801D9FF207047C0B270476F
:108030002DE9F041B1F9025000231E240F228542A0
:1080400003DDB1F90000BDE8F081B1F97A50854255
:1080500002DAB1F97800F6E701EB8205B5F90250D2
:10806000854201DA134600E01446E21852085D1C0E
:10807000AA42F1D101EB8203B3F90240844206DA4D
:10808000B3F9067031F92250B3F9046005E033F911
:10809000027C31F9225033F9046C001BC1178901AD
:1080A0003A1B41EA9061D3178001F8F73BF8721B45
:1080B000A0FB024601FB0261D31700FB03108106FF
:1080C00041EA9410284400B2BDE700002DE9F04FCA
:1080D000DFF8B8B16A48DFF8AC91DFF8ACA190F8EE
:1080E0000EC0BBF91A70BBF91C60BBF91850BBF984
:1080F0006C10BCF1070F48D2DFE80CF08D041A3089
:10810000485E7600D9F80020C284DAF800200285A3
:10811000C28C038DA7EB820212B2A6EB83034A4303
:108120001BB2594342F3CF2241F3CF23D11870E061
:10813000D9F800208284DAF800200285828CA5EB31
:10814000820213B2028D4B43A6EB820212B243F3BA
:10815000CF24514341F3CF23E11814E0D9F8002094
:108160000285DAF800208284028D838CA6EB8202DD
:1081700012B2A5EB83031CB24A43614342F3CF23FF
:1081800041F3CF24191949420AB244E0D9F800203A
:10819000C284DAF800208284C28C838CA7EB82022E
:1081A00012B2A5EB83034A431BB2594342F3CF22D9
:1081B00041F3CF24111914E0D9F800208284DAF8B1
:1081C0000020C284828CC38CA5EB820212B2A7EB82
:1081D00083034A431BB242F3CF24594341F3CF22D6
:1081E000A11849420BB216E0D9F800200285DAF84E
:1081F0000020C284028DC38CA6EB820212B2A7EBD0
:1082000083031CB24A4342F3CF23614341F3CF229D
:10821000991849420CB2BBF91E50594605F21E5638
:10822000A64201DACE8306E0A5F21E55A54201DD85
:10823000CD8300E0CC83B1F9204004F21E55954275
:1082400001DA0D8406E0A4F21E54944201DD0C8490
:1082500000E00A84B1F9222002F21E549C4202DAA4
:10826000ABF8224008E0A2F21E529A4202DDABF8BF
:10827000222001E0ABF82230417B8173BDE8F08F12
:10828000C00200203C2401403C2801405805002049
:108290002DE9F04704467B487C4E002702787A4857
:1082A000022AB0F9341004D0082A6ED0092A6DD001
:1082B000E3E0C27B022A02D1B0F844205AB1A4F80C
:1082C000421071810423B6F908101A460020FEF707
:1082D00001FF3081D1E06E49DFF8B881496A0D14A1
:1082E000E58090F84A1099B10089DFF8AC91C0F3AD
:1082F000C001C0F30020814223D1D8F8440040F2ED
:10830000BA41884240DD40F66A1188420ADC15E035
:10831000B4F9020040F2DA21884279DD40F26A4184
:10832000884204DD0823B4F942101A464EE0A0F258
:10833000DA20F8F780F80022584B56E0A0F2BA4055
:108340004FE057480078C0060CD5D8F8440041F2F9
:10835000243188425CDD41F2D4718842E2DC00F6CF
:10836000DC4020E04F48DFF8409190F87010012980
:108370000DD090F86F00012809D04C480178C9074A
:1083800046D04B49098889B142E06FE073E0B4F907
:10839000020041F6DC6188423ADD42F23411884243
:1083A00010DC00F59270A0F500501AE0B0F9100052
:1083B000B4F90210A0F59672914229DD00F596728B
:1083C00091420BDDB4F9421020231A460020FEF73B
:1083D00081FEA4F84200002817DB1BE0081A00F514
:1083E0009670F8F728F800224B46F7F790FF0E2218
:1083F000F7F7FCFFF8F756F800B2C0F58040684385
:108400008013A4F84200002D04DCA4F8427001E0BF
:10841000A4F842502748B4F84210F1804186264A19
:10842000818E318113782549012B10D0B1F912309A
:10843000D8F85010591A738B03EB6101F18209B21D
:10844000002900DCF782117839B1C08E0CE0B1F957
:108450001210B0F84630C91AEDE7B0F93600B6F997
:108460001610884200DB0846708106E01448B0F818
:108470007C00708100E07181378184F84070BDE834
:10848000F08700006F070020C0020020600000207D
:10849000580500205001002000C0924000007940A3
:1084A00040070020A40E002000C08240F80A0020EF
:1084B0001A000020780A002008060020100B002077
:1084C000600C00202DE9F041B1F9025000232B246B
:1084D0001522854203DAB1F90000BDE8F081B1F957
:1084E000AE50854202DDB1F9AC00F6E701EB820542
:1084F000B5F90250854201DD134600E01446E2184A
:1085000052085D1CAA42F1D101EB8205B5F9023097
:10851000834206DA35F9026C35F9044C31F9221040
:1085200006E01E4631F92240B5F90630B5F90410CF
:10853000801B091BC5178911AD0345EA90458703C8
:10854000A1FB070CCA1702FB07C201FB05219A1BFE
:10855000D317F7F7E7FD000A40EA0160001900B2FF
:10856000B0F5804FB9DB43F6FF70B6E770B5134C3A
:1085700040F224452946204600F02CF800281BD064
:10858000204600F046F82946204600F01DF80C4C25
:1085900000212046FAF7E0FA2046FAF75BFBC0F12B
:1085A00064000849C0B20428087201D900F0FCF93F
:1085B000BDE87040FAF78CBB70BD00000038014088
:1085C00058000240A40600200A0A01219140C94334
:1085D0000180704730B501F01F0201240025C1F36E
:1085E000421304FA02F2012B0FD0022B0FD0838A20
:1085F0004FEA11210088134204FA01F400EA040052
:1086000001D000B10125284630BD8389F0E7038AF7
:10861000EEE78088C0F308007047000070B5214C79
:108620002068214D400103D520492846F8F78EFDEA
:108630002068000104D51D492846FF31F8F786FD62
:108640002068C00003D51A492846F8F77FFD19486D
:10865000194A0178CB0712D192F82F30012B0ED096
:10866000F9F7BEFC2068C0F382611448072916D0D0
:10867000216811F0E05F01D15521017070BD012327
:1086800082F82F3021F0010101700D4801680D4A78
:1086900001F4E06111430160BFF34F8FFEE7002159
:1086A000EBE700000864004000640040010000386F
:1086B000000001386E080020180F00207808002004
:1086C0000CED00E00400FA052DE9F0478AB0002423
:1086D0004FF00408A34D8DF808804FF4806A009491
:1086E00001948DF80A408DF8134051462846F8F75A
:1086F0008DFE9D4E4FF0010901281CD186F83040B7
:10870000F8F7A2FC286840F400402860954814302F
:10871000016821F001010160944F386800F06EFE9D
:10872000002193A001F0E2FE386051462846F8F798
:1087300025FD86F8309002212846F8F767FE0128CB
:108740007ED16A4600212846F8F736FF01988B490A
:1087500020F0604088609DF80A1008294DD18849B2
:10876000421A88426DD00ADC864940180ED08649EC
:10877000401843D0012846D00728EFD14FE0012A06
:108780007DD0022A7CD0032AE8D1E6E09DF80B00D8
:108790001128E3D17D48406C322813DA7C48007BF5
:1087A000C0070FD000217B4800F0AAF97A4886F86C
:1087B0002F900168794A01F4E06111430160BFF331
:1087C0004F8FFEE7764A1121CDE905428DF81C80D6
:1087D00008228DF81D4003208DF81E208DF81F10F3
:1087E0008DF82000022005A90A18401CC0B2D472DE
:1087F0000828F9D32846F8F737FFA7E05F489DF827
:108800000B106F3074E05D4A0020694617320B1878
:10881000DB7A1354401CC0B20828F8D396E05749BD
:108820009DF80B204F311309087862F3030063F3BE
:108830000410530963F34510920962F3871001E0B5
:1088400088E02EE008709DF80C0048709DF80D003F
:1088500088709DF80E00C8709DF80F000A7960F3CB
:108860000002400860F347020A719DF81000487149
:108870009DF811208879930862F3010001E02DE052
:108880003EE063F38300120962F3071088719DF8DC
:108890001220C87962F30600D20962F3C710C871CA
:1088A00054E040489DF80B1001709DF80C10417089
:1088B0009DF80D1001F003028270C1709DF80E103A
:1088C00001719DF80F1041719DF8101081719DF894
:1088D0001110C1719DF81210017237E027489DF800
:1088E0000B205730017862F30101920862F387018F
:1088F00001709DF80C1041709DF80D10817016E00C
:108900001E489DF80B105F30027861F303020909DD
:1089100061F3071202709DF80C1041709DF80D1064
:10892000827861F30602C90961F3C71282709DF86B
:108930000E10C1709DF80F1001719DF8101041715B
:108940009DF8111081719DF81210C1710221284605
:10895000F8F714FC0AB0BDE8F08708489DF80B1042
:108960006730C5E700640040180F00207C08002035
:108970006465765F63616E3100000000900700203F
:108980000901FF18EEFF09EE11FFF6F85001002073
:10899000480C0020009003080CED00E00400FA05EC
:1089A0004200F6115C10002070B51D4D002428789F
:1089B000432834D16878462831D1A878502807D088
:1089C000512805D0812803D0892801D0212826D11B
:1089D000144E7071E9787172A81C891CF9F7C0FBFC
:1089E000B072717A294409793182884217D106F12F
:1089F0000E00017841F0020101700B48016841F05E
:108A000020010160317A0948002204E02B5D035502
:108A10002A55641CE4B28C42F8D38078707170BD22
:108A200030090020A40600200C0C0140DE0D0020BF
:108A300070B51D20FDF716F9FCF744FB1D20FDF76E
:108A400027F9154890F82F10144D0623144C85F87B
:108A5000381090F83B1095F83B201143012A04D0C0
:108A6000022A07D0042A0AD010E0827A8A420DD066
:108A7000007B09E0027D8A4208D0807D04E0827F8D
:108A80008A4203D090F82000884200D12370002051
:108A900085F8400070BD00007404002050010020E3
:108AA0006F0700200B4800214180A0F1B8018A899E
:108AB0008280CB891A44C2800B8A1A4402814B8A75
:108AC0001A444281898A1144818143F6FF71C18130
:108AD0007047000008020020084940F61C72B1F9F6
:108AE0000C00904202DA00F59F7005E041F2E302CB
:108AF000904201DDA0F59F70C881704760000020A2
:108B000070B50C460546FAF739FC3520FAF7AEFB8E
:108B10002846FAF7B1FBFAF7E3FBA4F57F41FF39EA
:108B20000FD0FAF72BFC3520FAF7A0FB2146284698
:108B3000FAF7FAFB0446FAF7D3FB042C01D0002025
:108B400070BD012070BD000038B51348C16941F007
:108B50000401C1611E208DF8000002208DF8010083
:108B60008DF8020001248DF803406846FDF79CF85B
:108B70000A4984200880094947F690602C31088012
:108B80000020091F0880054914310C80091F088046
:108B9000081F048038BD000000100240000800409B
:108BA00030B420491E4A45788B7A114692F83B40F2
:108BB00091F83910AC4218D14BB10379994202D0E7
:108BC0004379994201D140791AE0807909E08379AB
:108BD000994202D0C479A14202D182F82F3011E02B
:108BE000407982F82F0030BC7047C578AC42FAD18A
:108BF0006BB1C379994202D0037A994205D1007AC8
:108C000082F82F0030BCFEF70FBB407AE9E7437AC9
:108C10009942E2D00479A142DFD0007AE1E7000076
:108C20007404002050010020FEE700002DE9F04709
:108C30000446007F012868D13548E1880288511A2E
:108C400089B2072916D30088E080B4F9000044F205
:108C5000DD414843401346F6D96148438013A06084
:108C6000401000B2A0814FF08051B1FBF0F0F7F757
:108C7000DDFB2061B4F90C6096B1B4F902104DF639
:108C8000B05048430014A082B4F904704DF6B052BD
:108C900007FB02F24FEA2245E58204D4024603E0D4
:108CA0000020E08330E0424212B22283002D01DB3B
:108CB0002B4600E06B421BB2DFF858906383984666
:108CC0004FF4804AB24208DAF7F7A7FB2169F7F7B9
:108CD0007AFAF7F7CEFB801304E0002901DA484660
:108CE00000E05046E083B04509DA2846F7F795FBE7
:108CF0002169F7F768FAF7F7BCFB801304E0002F4F
:108D000001DA484600E050462084BDE8F0870000C4
:108D10007807002000C0FFFF2DE9F0414E484F4E7C
:108D200000250078A6F15004022806D14C4FF87BAC
:108D3000022802D1B7F8440030B1A5862564B56297
:108D400084F83850BDE8F08146488168C0684943DE
:108D500000FB0010FAF7D6FC40F233314843810B98
:108D6000B4F8440043F6CC42504301EB903080B25B
:108D700043F69911A4F8440088420DD33A481146AD
:108D8000B0F90400884207DB97F84A00032803D1B2
:108D900036480078012813D00123B4F934101A465C
:108DA0000020FEF797F9A086B4F84000012301B235
:108DB0001A460020FEF78EF920648003B06226E098
:108DC000B4F8460041F69A13A0F51852663A9A4252
:108DD00009D2B4F94400214AFAF716FB20640120B5
:108DE00084F8380022E044F24711884212D994F8FE
:108DF0003800D8B11E480178491CC9B20170022957
:108E000014D30570206C10B1401E206408E084F873
:108E100038500BE0A0F58040B0F5A47F03D2206C61
:108E20008003B06202E084F83850B562B4F84000C4
:108E30000A4980B20839323401F026FDB4F9000045
:108E4000B4F91810414389136180B4F916104843EE
:108E50008013A08076E700006F070020C80A00207A
:108E6000C0020020040A002010060020080600208E
:108E7000440100200D480021A32280F82810C1835E
:108E800081865030C2600E22028241F2620242614B
:108E900008220283418340F6386282839203C0E94C
:108EA00008124FF4B672826081627047780A00201F
:108EB0002DE9F0410546FAF71DFD204C204E0746EE
:108EC00020686168421C8A4220D009B93F281DD021
:108ED00004EB0010AA7A05F10B010E30F7F753F9F5
:108EE0002168686804EB011188602168A87A04EBA6
:108EF0000111888172B62068401C2060402801D38F
:108F00000020206062B6307888B114E03846FAF765
:108F1000D9FC0A28D4D3706800F070FA002109A0A7
:108F200001F0E4FA70604FF0FF30BDE8F0815520A9
:108F30003070F9F755F80020F7E70000F41400202E
:108F4000780800206465765F63616E310000000080
:108F500010B504000B462D4AC3F1000028D5644229
:108F6000002B12DAA04207DA214600F0F1FB32F8BA
:108F70001000C0F5404041E00146204600F0E8FB0B
:108F800032F8100000F5004038E0A34208DA21462C
:108F9000184600F0DDFB32F8100000F540402DE0EF
:108FA000204600F0D5FB32F81000C0F5803025E0F7
:108FB000002B12DAA04207DA214600F0C9FB32F892
:108FC000100000F5804019E00146204600F0C0FB8B
:108FD00032F81000C0F5004010E0A34208DA214644
:108FE000184600F0B5FB32F81000C0F5804005E0EF
:108FF00053B1204600F0ACFB32F81000B0F5004F42
:1090000001DDA0F5803010BD002010BD80BD00083E
:1090100040438013494300EBA13000220302002BA0
:1090200014DDB3F5001F01DC802001E04FF4005097
:1090300093FBF0F1014401EBD1714910814206D05C
:10904000521CD2B20846062AF2D300E00021C80022
:1090500000B2704702E008C8121F08C1002AFAD106
:1090600070477047002001E001C1121F002AFBD1A8
:10907000704700002DE9F047BD4CBE4821880288AA
:10908000511A89B20F297DD30088A4F13C052080B4
:10909000288F08B1401E28872B78B74AC3F3810078
:1090A00001281ED0022821D0118BB148B44EDFF820
:1090B000CC92407EB6F806C00027B1F5926F1CD85E
:1090C000142818D3782060764CF01000F08040F21D
:1090D0006660A88123F001002870D77389F80070BA
:1090E00018E0108B00EB4000C00302E0108BA54994
:1090F0004843010CD9E7401C04E0B1F5216F09D9C0
:1091000010B1401E607605E02CF01000F08043F0B6
:1091100001002870B5F90200B5F914304143C3EBE2
:10912000C303C1F38F31C3F3D10303EB510109B280
:10913000A9829046128B4FF080535043B5F9162008
:10914000C0F38F30C2EBC202C2F3D10202EB500077
:1091500000B2E882AA6A42431213EA6293FBF2F277
:109160002A63894A1080A2680A44A260E168014427
:10917000E160207C401CC0B22074072802D942F371
:10918000CF0000E0E8E02883C9106983E760A760AA
:1091900041F6C8012774884204DD2A8B7B49B1FB64
:1091A000F2F1E981C117890341EA9041800342F657
:1091B0009B420023F6F7B6FFA8846D482A78A0F1F9
:1091C0003C009307B0F90600C2F3810200EB801166
:1091D00001EB003141F30F3115D5012A07D0022AE6
:1091E0000BD04EF6AC3141430914A18011E049F295
:1091F000586250430014A08020E04CF20C314143EF
:109200000914A18026E0012A0ED0022A18D0A080DD
:1092100069845F4948430014A4F81E00F9F7DAFE98
:109220005C480088C0B143E04AF2904242431214C5
:10923000A2804BF2C822504300146884E183EDE71A
:109240004CF6345141430914A1804DF66C31414331
:10925000091469845049DDE795F8200000BB88F8BF
:109260000F7089F80070B5F91A00A0F514512C3967
:10927000B1F56E7F18D2617FF42912D94749E88091
:10928000434AA1F8460050430014A880A1F84400C6
:10929000FF2085F8200081F8280041493C20087013
:1092A00006E0491C617703E0607F08B1401E6077EB
:1092B000B5F91A00B4F91E203A4990420DDDA27E9C
:1092C0007D2A08D9F28842F00802F2800A7822F05A
:1092D00002020A700EE0521C06E0A2F23D12904219
:1092E00008DAA27E12B1521EA27603E0F28822F0C2
:1092F0000802F280B4F90420904214DA2A4B9B68E9
:10930000B3F5FA7F0FDAE07E3E2809D9F08840F005
:109310001000F0802777087820F0020008700CE039
:10932000401CE07609E002F23D12904201DD88889F
:10933000A0B1207F08B1401E2077B5F918106069F0
:1093400008446061217E491CC9B221761F2903D9D6
:109350004011A88367612776BDE8F087207F7D28CC
:1093600004D9F08820F01000F080E6E7401CE3E725
:109370002805002078070020C00200206F07002089
:10938000480C002030330100B80B002074E8260B95
:10939000188601007A070020E0380100A40E0020A2
:1093A0006C0700201006002058050020024941F2F9
:1093B000F460886270470000EC04002070B50D4C2A
:1093C000207828B1012808D0062505280FD10BE008
:1093D0000948F9F7D5F8012004E00748801DF9F79E
:1093E000CFF80520207070BDF9F7EAF825702570D8
:1093F00070BD00007007002088BC00080A4A4FF0CA
:10940000FF31B0EBA20F0CDA00280ADB074909682C
:1094100051F820004068006900B100476FF0050076
:10942000704708467047000004000000AC080020A8
:1094300070B50A4DA86870B100240948AC60F7F710
:109440002DFF084804604460A0F58160046044601A
:109450002C70002070BD6FF0040070BD78080020F3
:1094600000640040F41400207FB505460024631E0C
:10947000244A4FF00050072D41D2DFE805F04004A8
:10948000111E21403C00814208D2D068202805DA14
:109490001D4B43F82010401CD0600CE01C4627E018
:1094A0008142FBD210692028F8DA174B803343F849
:1094B0002010401C10610023F0E7F7F705FF17E0CC
:1094C00000208DF80B000121ADF800000422ADF85A
:1094D0000400ADF808008DF80C108DF80A00ADF806
:1094E0000220ADF806208DF80D106846F7F728FF2A
:1094F000204604B070BDBDE87F40FAF78FBA184629
:10950000F7E7000078080020FC180020F8B5414E6D
:10951000B06801287BD04048F7F7C0FE0121082041
:10952000FCF786FF01210846FCF782FF012148066F
:10953000FCF766FF01214FF4EA10FAF787F94FF4C0
:109540008070ADF8000003248DF802400420334DF4
:109550008DF8030069462846FAF726F96815ADF834
:1095600000008DF8024018208DF803006946284657
:10957000FAF71AF914208DF8000002278DF801700F
:1095800000248DF8024001258DF803506846FCF751
:109590008BFB13208DF800008DF801708DF80250C0
:1095A0008DF803506846FCF77FFB16208DF800000D
:1095B0008DF801408DF802408DF803506846FCF7A5
:1095C00073FB17490120FFF74FFF16490120FFF7F2
:1095D0004BFF15490120FFF747FF14490120FFF712
:1095E00043FF13490120FFF73FFF00210320FFF74E
:1095F0003BFFF7F7FFFD0F4804604460A0F5816072
:109600000460446034700020B560F8BDFFE74FF09F
:10961000FF30FAE77808002000640040000C0140A9
:1096200020FF401820FF431820FF441820FF451852
:1096300020FF2518F41400202DE9F04781461E482C
:1096400086B0174680680E46A0B14FF0FF381FB3B2
:109650006846FAF7F1F9401C0ED00DF10B019DF8A8
:109660000A208A464846019DF6F78DFD9DF80A407E
:109670003D601DE06FF0040006B0BDE8F08700BF5C
:10968000FAF7CCF9411C15D0A84213D16846FAF775
:10969000D3F90198A84201D04046EDE79DF80A2091
:1096A00009EB04005146F6F76EFD9DF80A000444EC
:1096B000B442E5D32046DFE7780800202DE9F047E3
:1096C0000646224886B00024806888B1601E002AC1
:1096D00010D012680192B2F1005F0BD2CF0801F0F6
:1096E00007054FF000084FF004094FF0080A17E093
:1096F0006FF0040006B0BDE8F08700BF8DF80AA047
:109700008DF8089006EBC4008DF809800168CDF84B
:109710000B104068CDF80F006846FFF7C9FB641CCA
:10972000BC42EBDB7DB18DF80A508DF808908DF8C6
:10973000098006EBC4012A460DF10B00F6F723FD64
:109740006846FFF7B5FB0020D4E70000780800204A
:10975000090A05D0B0FBF1F0FF2800D9FF207047BF
:1097600000207047D0E90021C368521A5A4301EB28
:10977000A231816041607047B0F90020B0F9021059
:10978000B0F90630521A5A4301EBA2318180418070
:109790007047000030B5494B18884949CA8A801A79
:1097A00085B24848484A0F2D047801F158001DD36E
:1097B0001D88CD82117A090713D5022C01D04349A7
:1097C00012E0434DB0F90210B5F90050A94205DC92
:1097D00002DA01F1020108E0458007E0A1F102018F
:1097E00003E0022C02D13B4909884180B0F84010C7
:1097F0001D88691A89B29C2949D31988A0F840109C
:10980000D16A0023B1F5804F31DB3349096DB1F5E1
:10981000405F2CDD314940F26665B1F91010A94274
:1098200012DD43F69915A94202DB40F2333108E01C
:1098300040F23335A1F26661694343F2333591FB5F
:10984000F5F1A0F8441001E0A0F844302449B2F842
:109850000A510978C1F381012DB100BFB0F844105D
:1098600001F21E511CE092F84A20032A10D0A0F801
:109870004430022C01D0A0F84430B0F95C10B0F9AB
:10988000443001F114029A420DDAA0F85C2030BD98
:10989000012901D00229E1D1B0F8441001F233319D
:1098A000A0F84410E5E703F11402914203DD1439F6
:1098B000A0F85C1030BDA0F85C3030BD7807002007
:1098C000080000206F070020C0020020EA040020EA
:1098D000E8040020E4040020500100205805002086
:1098E000EC0400202DE9FC4101210220FCF788FD59
:1098F00001211920FCF79CFD01213C48F9F7A6FF46
:109900004027ADF8007003248DF802400420384D44
:109910008DF8030069462846F9F746FFE001ADF8E7
:1099200000008DF802401C208DF80300694628468F
:10993000F9F73AFF4FF4E0712846F9F7BCFFA81594
:10994000ADF800008DF8024010208DF80300694644
:109950002848F9F729FF4FF4A060FCF7D7F91D203C
:109960008DF8040001268DF8056000258DF806505D
:109970008DF8076001A8FCF797F91F498C20088033
:109980001D494FF6FA702C3108806E20091F08809F
:1099900019481430068018480830078016492031CD
:1099A0000D80154AD020121D1080134A45F2F30095
:1099B000183210800A1F45F2500010800E4A4FF6F0
:1099C000FF7038321080121D1080121D108041F27D
:1099D0001B10088000F012F8FAF758FC0648103007
:1099E0000580001F0480BDE8FC810000000C1A0007
:1099F00000100140000C01400004004070B51D2023
:109A0000FCF725F92B4D4FF480712846F9F74AFFF2
:109A1000840080212846F9F745FF44EA40044021AC
:109A20002846F9F73FFF0443E0B2234C84F83C009A
:109A3000F9F7E2FF0546052805D92048C18841F01D
:109A40004001C18001E084F838501D48007A0007C9
:109A500003D594F838001B490D5C4FF6FA7020636B
:109A6000E062A06260622062E061A061164860630B
:109A700000206064206584F83F0084F84000F9F716
:109A800069FFA07AFF2812D05FF0020084F83D0041
:109A90000E480088A0662846FAF772FE207820F06B
:109AA00001002070BDE870401D20FCF7E6B80120E1
:109AB000ECE700000010014050010020480C00209D
:109AC000C00200207CC60008DCFF05002404004022
:109AD0002DE9F00F5848594902880B889A1A92B21A
:109AE0000F2A7DD30988DFF858910180B9F81E103C
:109AF000027D00EB42029180017D491CC9B20175D3
:109B000008296DD3002404752246017D00EB410332
:109B1000491CB3F90430C9B202EB630212B20175F9
:109B20000829F2D347490475474B4A8044800E7890
:109B3000DD895FEAC67C40F6386A4FF0030714D02F
:109B4000A2F22B5C42F6E858C44520D3A1F1080CE0
:109B500026F00204ACF8062047750C7040F22B5436
:109B6000A24211DA45F0040222E046F001060E702E
:109B7000524507DD45F00102DA8126F002020A7043
:109B800047751BE0447519E045F0020210E05245AC
:109B900010DA8775427D12B1521E42750EE046F012
:109BA00002020A70DA8822F08002DA8025F00702C9
:109BB000DA8103E0837D3BB15B1E8375408888803A
:109BC000BDE8F00FFCF7B6B842F6AA239A422BDAAA
:109BD000B1F904503DB941F2CD039A4203DA00E0F5
:109BE00026E04480EAE7194B920302EB833241F608
:109BF0007243B2FBF3F212B2428099F80840034676
:109C0000240702D540F2333401E040F69914A24211
:109C100000DA5C80B3F90220521B02F5A372B2F5A0
:109C2000237FCBD85D80C9E74FF480434380C5E7ED
:109C3000BDE8F00F70470000E00C0020780700201E
:109C4000C002002010060020480C0020C8F1FFFFD1
:109C50002DE9F0416D4CDFF8B8E14FF0000594F8C4
:109C60003410C80706D094F938104B42002958DD4B
:109C70000E4657E0674884F83750A4F84250664AC9
:109C800090F8380084F840009586CEF80450CEF85D
:109C90000850624E40F26663CEF80C50A4F87C3057
:109CA00036F810005E4E768830444FF6FF7606EAAE
:109CB000800024F8300B4FF0806044F8040CA3209F
:109CC000208460845810A084E38440F69910208595
:109CD000580060854FF48050A08541F23330E08514
:109CE00041F26660208641F69910608641F6CC40CC
:109CF000A0864FF40050E08642F23330208742F2D3
:109D00006660608742F69910A08742F6CC40E087F3
:109D100082F8A15041F00100207184F84450BDE860
:109D2000F0811E4694F937004242002801DD0746C3
:109D300000E01746F61B012E0BD0002800DB024680
:109D40005FFA82F684F8380094F84F00012805D0B5
:109D500041E0002900DA1946CEB2F3E794F9393030
:109D60005942002B01DB184600E0084694F93A20DE
:109D7000C7B25042002A01DB944600E08446BC454D
:109D800008DD002A00DA0246D7B2002B00DA0B46C3
:109D9000D8B207E0002B00DA0B46DFB2002A00DB66
:109DA0001046C0B204EB4000B0F9501004EB47007D
:109DB00030F9502F11444910018084F84F5084F835
:109DC0003E5084F83D5084F83C5084F83B5084F871
:109DD0003A5084F8395004EB46007546B0F950000B
:109DE00024F8420FBEF80410C82309B26422FDF71C
:109DF00071F96860E968401AA9680844A860B5F973
:109E000000104843C013E860608788E7600C0020BA
:109E1000F805002050010020C00200208EC6000876
:109E200060000020F0B4544890F83410C90776D090
:109E3000524990F84030002291F838108B426FD090
:109E40004F4CA0F872204F4DE65C04468E4294F9C8
:109E5000374002D0EE5C8E420FD1641C64B280F8B1
:109E60003740EB5C8B4202D1641C80F8374090F99C
:109E700037300F2B1BDD0F2317E0434DEE5C434DB6
:109E80008E4202D0EE5C8E4211D1641E64B280F824
:109E90003740EB5C8B4202D1641E80F8374090F96A
:109EA00037406FF00E039C4201DA80F83730324BB6
:109EB00090F83F50393390F83740EC5490F83F30E9
:109EC0005B1CDBB280F83F30062B01D380F83F20CB
:109ED00090F9394090F93B309C420ED190F93D40C9
:109EE000A3420AD190F93A4090F93C309C4204D107
:109EF00090F93E40A34200D1012280F84F201F4A32
:109F000080F8401090F937501378214A012D0DDD6B
:109F100014465E07A46804D544F0080403E028E072
:109F200015E024F00804946080F83510B5F1FF3F87
:109F30000ADA5B07936802D523F0080301E043F0D7
:109F40000803936080F83510F0BCF9F703BD90F872
:109F50004F1001290DD1B0F8721043F60953491C76
:109F600089B2A0F87210994203D9A0F8722080F843
:109F70004F20F0BC70470000600C00205001002012
:109F800070C6000876C6000882C6000888C60008A9
:109F9000C002002010B502884188B0F90830114491
:109FA00009B281FB0313890B428041EA8341B0F976
:109FB0000420B0F9063082FB0332940444EA933261
:109FC0001144818010BD000030B52049204AB1F80D
:109FD0006A301088C01A80B20F2836D31088A1F8D2
:109FE0006A001C4D00204FF000432A5C940903D006
:109FF0000124B4EB921F24D1D20622D0164A52F883
:10A0000020201268134C123434F81040224201EB25
:10A01000000494F9722008D00A2A04DB0A6823FAA3
:10A0200000F4224308E0521C09E012F10A0F05DC9B
:10A030000A6823FA00F4A2430A6002E0521E84F880
:10A040007220401CC0B21128CFD330BD18060020AA
:10A050007807002084C1000884C200082DE9F007B9
:10A060007A497B480A8903889A1A92B2082A75D3DA
:10A0700000880881A1F12C0042890AB1521E428158
:10A08000744A92F82820802A68D302F03F020A70AE
:10A09000C2890AB1521EC281B1F90620902A0CDB96
:10A0A0008A46FF2A09D08146C089002856D16A48CD
:10A0B00000230078092805D005E0BDE8F0076348D3
:10A0C00000F0C6B90823654A92F8EE500DB143F08E
:10A0D00004036348017BC90701D043F00203D2F8AF
:10A0E00008C05FEA0C5101D543F001031768002155
:10A0F0005C4EFC0302D596F8654004B18021C4880B
:10A100005FEA446801D541F040015FEA845801D517
:10A1100041F020015FEAC47801D041F01001807A5B
:10A12000400701D541F008014F480078C00701D031
:10A1300041F00401A00601D541F001010020012DEC
:10A1400000D1082096F870508DB992F84A20032A61
:10A1500005D0022A06D0012A07D008E072E040F0BC
:10A16000030004E040F0020001E040F001007A0743
:10A1700001D440F02000CCF3C0020025CCF3002C29
:10A18000624502D13A0700D4042596F86F20012ACF
:10A1900001D145F00105354A0027BC4612783E46FC
:10A1A000C2F38102012A04D0022A04D0032A04D077
:10A1B00004E0022602E0042600E010262C4A640691
:10A1C0000ED5224C1C342478240609D51478640654
:10A1D00006D4284A40F6CC44926D6243140C05E044
:10A1E000B2F8B62040F699146243940B4FF0080879
:10A1F0008AF80A804FF061088AF80B808AF80C30E0
:10A200008AF80D108AF80E008AF80F508AF810703C
:10A21000270A4B4083F06901414069408AF8117078
:10A2200079408AF81240614052468AF813C0714062
:10A230008AF8146051754FF4C871A9F80E10FF2008
:10A24000AAF80600BDE8F0077047000024070020C8
:10A2500078070020180600206F070020C0020020A9
:10A26000480C0020A40E0020F80A0020EC04002076
:10A270005001002094090020FBF7B2FD5D48816980
:10A2800041F0FC0181614FF4A060FBF73FFDFAF75C
:10A29000A3F8F6F7C3FCFBF71BFB002156A000F068
:10A2A00025F958490860FDF71FF8FCF719FEFFF77C
:10A2B00019FBFAF781FFFFF7A1FBF9F7E7FF00F0C1
:10A2C00009FC514D4FF40050A5F81A014F48407851
:10A2D000FF2801D0FBF754FFFBF708FF00214FF4E4
:10A2E000FA5340F2EE220020401C80B29842FBD389
:10A2F000491C89B29142F6D34548002680F8726025
:10A30000F6F71CFBF8F72EFAF7F736FFFEF71CFC02
:10A31000102240494048F5F736FF01F02BFB3F4C37
:10A32000404FE08820F04000E0803D48017821F077
:10A3300020010170FA20F8814FF49670A5F84200D0
:10A34000FFF734F838493948FBF77BFE3848FBF70C
:10A350009DFE3848416A88473748416B8847FEF779
:10A3600089FD3648F8F732FEF7F738FF34494220C6
:10A37000C8803449C8603448F6F710FEA86820F455
:10A380008070A86031483E71017841F08001017011
:10A39000E088208260896082A089A082F9F766F94E
:10A3A000F9F7C2F8FEF766FE01F064FAFFF790FBDA
:10A3B00000F038FAFFF708FE01F0FEF8FDF7F4FDB3
:10A3C000F7F736FFFAF7FAF9FFF7E4F9FCF7C0F808
:10A3D000F9F70CFCF9F73EFC00F0B6F8FFF73EFE8B
:10A3E0001648F8F79FFC00F095FBFCF7BDFDF8F769
:10A3F00023FECDE7001002406465765F63616E3135
:10A40000000000007C080020C0020020007003084B
:10A4100058050020A40E002058060020480C0020FB
:10A42000500100206C070020480A0020180A002074
:10A430002804002034000020E0000020840B0020CD
:10A44000600700205C040020F80B0020400700207B
:10A45000F0B523490278B0F9064000231F4E31F8C9
:10A460001210FF2C18D0B0F904701E4DBC4231DA26
:10A4700000EBE40704F00704BF7AA7408478FFB23A
:10A480003CB190F801C0ACF1010C64451FDA3C0608
:10A490001DD455F822200DE056F8222011601249F3
:10A4A0008A79521CD2B28A71022A02D38370C38085
:10A4B0008B71F0BD11608178491CC9B281704278FE
:10A4C0009142F6D38370C188491CC180F0BD56F813
:10A4D0002220EFE755F822201160F4E764C300085A
:10A4E00096C100080CC30008F80600202DE9F041D1
:10A4F0000F4680460024124D124E08E0286850F89E
:10A50000240001684046F5F750FE38B1641CB4EBF6
:10A51000A60FF3DB6FF00100BDE8F081286850F86A
:10A5200024004068016829B13846884728B16FF097
:10A530000200F1E76FF00500EEE72046ECE70000CF
:10A54000AC08002004000000F0B561486149B0F893
:10A550006C200B889A1A92B29C2A7BD30988A0F8A7
:10A560006C105D495D4F91F82A1001F0070297F8D1
:10A570004A10022A00D1491E594C80F83E104FF073
:10A580000203E2884FF00001550401D5012236E0B4
:10A59000E489E50601D5062231E0250701D5082228
:10A5A0002DE0550603D44F4D2D78AD0601D504227C
:10A5B00025E0150501D5072221E0150601D50A225F
:10A5C0001DE0950601D50C2219E0150701D50B22D7
:10A5D00015E0550701D4D50501D510220FE0D506A9
:10A5E00001D505220BE0650703D4A50701D4E407D4
:10A5F00002D080F86E3007E0920403D5032280F881
:10A600006E2001E080F86E10374A384C92F820E056
:10A61000324A251FD2F808C02D4AB2F87060721C69
:10A6200092B2BEF1000F0DD02CF4000CC7F808C098
:10A6300090F86E70B7B11E2F1AD090F86F200AB341
:10A6400025E007E04CF40006BE60A0F870200A2A5E
:10A6500001D22360F0BD142A01D22B60F0BDA0F816
:10A660007010F0BD2B60A0F8701080F86F10F0BD76
:10A67000642E04D2A0F87020322AEED3E9E7A0F8C5
:10A680007010EAE77F1C80F86F70A0F8701090F8E7
:10A690006F20012A10D0002AE9D0B0F87060761C33
:10A6A000B6B2A0F870601E2ED7D323603C2EDED940
:10A6B000521E80F86F20D2E7B0F87020521C92B280
:10A6C000A0F870202360C82AD1D980F86F10C6E79F
:10A6D0001806002078070020A40E0020C0020020E9
:10A6E000480C002050010020EC040020141C014004
:10A6F000F0B54548B0F84810491C89B2A0F8481098
:10A7000002297DD341490024A0F848400A78404BF3
:10A71000042A5BD04FF48041082A0BD0A0F110022C
:10A72000B2F900208A4200DA1146B3F984208A4245
:10A7300000DA1146374A12698A4200DA11B24182C0
:10A7400082881D8AC2EB8502334D12B22D78C5F383
:10A7500081062D4D40F686567243B5F97650921219
:10A760006A431213C26086681546C6EBC60642F3FA
:10A77000D102F60202EBA6328260C66C1644C664B1
:10A78000B0F850707F1CBFB2A0F85070B7F5806F62
:10A7900004D3B6120682A0F85040C464C66A891A6F
:10A7A000A6EB461740F2545207EB07174A43A7EBB4
:10A7B000C61602EB4602466A32444262B3F93430AE
:10A7C000B2EB034F06DD1A04426206E01349B1F909
:10A7D0000410AFE7002A00DA4462C162104990F821
:10A7E0003D2091F838108A420DD080F83D10B0F825
:10A7F0004210A0F84410B0F84010A0F8421000E059
:10A8000001E0A0F84050F0BD580500206F0700207F
:10A81000C0020020440E0020EC040020580E00204E
:10A820005001002015481649B0F85A200B889A1A92
:10A8300092B20F2A20D30988A0F85A10B0F900105C
:10A840004FF48042C1EBC12141F35131A0F86C10AB
:10A850000C490B78A0F11001022B06D1B1F90030A0
:10A86000934202DA1B1D0B8000E00A800021A0F851
:10A87000601020F85C1F42807047000058050020DF
:10A88000780700206F0700204FF6FF7202EA80026F
:10A8900010F4404315480ED0B3F5804F14D0B3F5F3
:10A8A000004F4FEA122216D0C2F5807330F81330F1
:10A8B0005B424B8005E0120A30F812304B80C2F543
:10A8C000807230F812000FE0120AC2F5807330F87F
:10A8D00013304B8005E030F81230C2F580725B42D5
:10A8E0004B8030F8120040420880704780BF00085B
:10A8F000104A518AD08A928A16384639A2F111023A
:10A9000000D54942002A00DA52421144002800DAF8
:10A9100040420844084943F6284300B2B1F93620C2
:10A920005A43921340F2D733584302EBA030C88603
:10A9300070470000C0020020580500202DE9F043B8
:10A94000DFF88491614CB9F91C602663B9F91E5097
:10A950002564B9F94C202260B9F94EC0C4F81CC076
:10A96000D4E9051041438F136168E368521AD21A83
:10A9700023695A4307EBA2326261E76AD4F8288060
:10A9800078438713206A921BACEB000CACEB080CED
:10A990000CFB03FC07EBAC33E362A3EB050363643E
:10A9A000626301D4944601E0C2F1000C474DE66BAE
:10A9B000AD6B6F42B44504DA6A4392FBF6F2E26093
:10A9C00004E0002A01DDE56000E0E760002B1A46A4
:10A9D00000DA5242B24204DA5D4395FBF6F2A2621B
:10A9E00004E0002B01DDA56200E0A762E268531AD3
:10A9F000A26C534301EBA3316160A36A1B1A53435A
:10AA000000EBA3302062A368CD1A554303EBA533B6
:10AA1000A360636A4942C51A554303EBA53209B2E4
:10AA200000B26262F7F70EFB294D28802089404270
:10AA300001B2A08C00B2F7F705FB68802988E164B9
:10AA4000B9F83A20531AAB80101AE880206D081A22
:10AA500010F5004F03DC00F58030E26D05E0E26D9B
:10AA6000B0F5004F01DBA0F5803010442165E065B2
:10AA7000206E401C20660A2804D1E06D606500202D
:10AA80002066E065D4E91510091A00EB211045F69F
:10AA90008E3180FB0112890BA06551EA8241E1668B
:10AAA00000D54942A166002800DA404243F2333122
:10AAB0004843C013A064642801DA6420A06440F213
:10AAC0006C70A064BDE8F083600000209409002051
:10AAD000000000200E4843F60951816140F6945170
:10AAE000016143F2846181634FF40051C1636421C9
:10AAF00081640021C16081624161C162C1644165BC
:10AB00008165C165016601658166C16670470000A7
:10AB100094090020F0B5904990480A8903889A1A50
:10AB200092B23E2A1ED30088088101F138004FF40A
:10AB3000FA63428A9A4202D2521C428200E0438265
:10AB4000874A92F82220802A0CD302F03F020A7032
:10AB5000B1F90620402A06DBFF2A04D0C2883AB1A8
:10AB6000521EC280F0BDBDE8F0407B48FFF770BCCC
:10AB7000428A9A42F6D307784FF0010E3A074FF017
:10AB8000FF055BD5847A40F2DC52630708D444F0B9
:10AB900004038372C28081F80BE081F80AE04CE084
:10ABA0004378072B05D0032B03D0052B01D0062BB0
:10ABB00007D1660605D444F040038372C2800522A3
:10ABC00039E0654A5FEA437C02F138024FF42076AF
:10ABD000127A0DD55FEAC26C0AD45FEA446C07D4DE
:10ABE00042F0100202723A0628D4C680192222E0EE
:10ABF000DF0709D0970707D4670605D442F00202A1
:10AC00000272C680042216E09F0709D5170707D4F1
:10AC1000670605D442F008020272C68003220AE0E9
:10AC20001B070BD5530709D4630607D442F004026F
:10AC30000272C6800B22CA728A72CD80494AB2F96A
:10AC40002230B2F91A7003F23D140022A74200DB51
:10AC50000276414E444C06F13806A479B6895FEA83
:10AC6000C46C06F101064FF4C874B6B213D58681E0
:10AC7000B6F57A7F05D9017A21F0800101728281CF
:10AC8000F0BD037A1E06FBD4828143F0800202727B
:10AC9000C480112035E09F4216DA037E052B13D2C3
:10ACA0008681B6F5487F04D98281027A22F040027B
:10ACB0000272027A5606E3D45B1C037642F040022D
:10ACC0000272C48002201CE0284B1C89C4F3C00619
:10ACD000C4F3002740F2EE24BE4216D11E78360798
:10ACE00013D4427E012ACBD1428BB2F5167F02D219
:10ACF000521C4283F0BD827A42F002028272C4800A
:10AD00000F20C8728872CD80F0BD93F811714FF496
:10AD10000046012F18D1164F41F6583C7F6C67450D
:10AD200012DD83F810E1134B1E60C38AA34202D2E6
:10AD30005B1CC382F0BD4FF4FA73C3801C23CB723B
:10AD40008B72CD80C282F0BDC2820A4883F8102186
:10AD5000001F0660F0BD00000807002078070020F3
:10AD600018060020EC040020480C0020C00200203F
:10AD700050010020140801402DE9F05FFE48037ED9
:10AD8000FE48011D0A1DFE4C012B5BD0B4F85E305D
:10AD90000380B4F860000880B4F862001080FDF70A
:10ADA00095F9DFF8E083F84D49F2CD32B8F91E107D
:10ADB000A983B8F9200043F6CC4C01EB4000504386
:10ADC0000014E883B5F92260B5F9203000FB06F2E3
:10ADD00001FB032242F38F326A82B5F9187058439F
:10ADE00007FB0CF740F2333CBF1302FB0CF207EBFE
:10ADF000A23201FB16002A8340F38F30A882B5F9F6
:10AE00001A1043F6AE72514300EB0012891302EBA5
:10AE10008010DE4F01EBA030DD4E6883786C30602F
:10AE2000316930468847DB49308948800846FDF75C
:10AE30002FFAF8F78DFFD84E4FF0010A4FF00009B6
:10AE400048B10DE0B4F864300380B4F866000880BF
:10AE5000B4F86800A2E73078082805D0688F288207
:10AE6000307804282AD012E0CC4890F93710491CD9
:10AE7000022921D890F8741019B1B5F85A00288227
:10AE800005E0698F2982A5F85A1080F874A0B5F9F9
:10AE90001410B5F90A00C24AF7F7E8FDE862B4F900
:10AEA0001A11884204DDBE48E962027C9140816249
:10AEB0003078042816D00CE0688FE0E7D8F824003A
:10AEC0000014E862E07B04280CD0C5F82C9086F8CA
:10AED0000090B34AB5F91210B5F90800303AF7F707
:10AEE000C5FD02E0B87AE8B3AE48AD4EA862443E74
:10AEF000AB463060E86A706030461035FBF704FB03
:10AF0000A14928883C39FFF7BFFCDFF87C82A8F113
:10AF10005808D8F81C10C8F87810B5F91010B068A7
:10AF2000B5F9122000FB01F7F368504303FB1276DA
:10AF300046F38F3703FB0100AF8740F38F36EE8770
:10AF4000994D28466F80AE80FDF770FE287F08F18E
:10AF50002005012834D0704241104DF6B35069806D
:10AF6000474300E029E03A142A808B18A8F80660CD
:10AF7000A8F80830B1EB0201A8F80A1084F80C9088
:10AF8000B8F90630002B01DD84F80CA0B8F90800F0
:10AF9000002802DD217B891C2173B8F90A20002AD0
:10AFA00002DD217B091D2173217B072923D2DFE8E4
:10AFB00001F0221E351B312033004FF4AF7094E7AF
:10AFC0007948B0F9203059424A106A80B0F91E0021
:10AFD0004DF6B351484301142980A8F806305318A0
:10AFE000A8F80830511AC7E784F80DA003E0022141
:10AFF00000E0032161739BF800106C4E01296C4F37
:10B00000617B0DD007297DD2DFE801F07CFDFCFBE0
:10B01000FAF9F8000421EDE70521EBE70621E9E75D
:10B020000729F0D2DFE801F06E04295D84D8F00032
:10B0300001461846FAF7ECFF2860B5F9020040F621
:10B040008151484380136880B5F9001040F6815261
:10B050005143891329804218A2F68152B8F814305E
:10B060005242C3EB620212B2A8F81220002A01DC9D
:10B07000A8F81290B8F812205AE1404201B25042AA
:10B0800000B2FAF7C5FF2860B5F9020040F6815119
:10B09000484381136980B5F9000040F6815250435E
:10B0A000801328800A18A2F68152B8F81430524250
:10B0B000C3EB620212B2A8F81220002A01DCA8F841
:10B0C0001290B8F81220A4F862201144A4F85E107F
:10B0D000084461E13046F5F7FFFD01231A460721D8
:10B0E000D9E019461046FAF793FF2860B5F9020037
:10B0F00040F68151484380136880B5F9001040F64E
:10B10000815200E0D2E05143891329804218A2F60F
:10B110008152B8F814305242C3EB620212B2A8F85E
:10B120001220002A01DCA8F81290B8F8122059E188
:10B130005942404209B200B2FAF76AFF2860B5F9F5
:10B14000020040F68151484381136980B5F900003F
:10B1500040F681525043801328800A18A2F681528B
:10B16000B8F814305242C3EB620212B2A8F81220AF
:10B17000002A21DC1EE00000840B0020342C01405A
:10B18000C00200205805002060000020500100206F
:10B190005C040020180400206F070020600C0020D1
:10B1A000480A0020A2FEFFFFB80B00200024014047
:10B1B00000280140A8F81290B8F81220A4F85E20E8
:10B1C0001144A4F86010084442E13046F5F784FDCC
:10B1D00001231A4605215EE01146FAF719FF28609F
:10B1E000B5F9020040F68151484381136980B5F9F1
:10B1F000000040F681525043801306E061E135E1E2
:10B2000006E1D7E0A8E07BE018E028800A18A2F663
:10B210008152B8F814305242C3EB620212B2A8F85D
:10B220001220002A01DCA8F81290B8F81220A4F825
:10B2300060201144A4F85E10084434E1504201B289
:10B24000584200B2FAF7E4FE2860B5F9020040F671
:10B250008151484381136980B5F9000040F681525D
:10B260005043801328800A18A2F68152B8F814308F
:10B270005242C3EB620212B2A8F81220002A01DC8B
:10B28000A8F81290B8F8122035E13046F5F724FD01
:10B2900001231A4606213846F5F71EFD01213046E6
:10B2A000F5F790FC01213846F5F78CFCBF4DBBF853
:10B2B0000810D8462980BBF80A106980BBF8100036
:10B2C000A8802846F7F790FDB4F95E60E88840F65C
:10B2D000815C304400B2A4F86400B4F9603029897C
:10B2E0006045194409B2A4F86610B4F962206F8968
:10B2F00017443FB2A4F868707EDDA4F864C012E180
:10B3000001461846FAF784FE2860B5F9020040F6B7
:10B310008151484380136880B5F9001040F681528E
:10B32000514389134218A2F6815252422980521089
:10B33000A4F862201044A4F860000844A4F85E0059
:10B3400000213046F5F73EFC00213846F5F73AFC7F
:10B3500001231A460621BDE6404201B2504200B226
:10B36000FAF756FE2860B5F9020040F681514843CD
:10B3700080136880B5F9001040F68152514389135B
:10B380004218A2F68152524252102980A4F862203B
:10B390001044A4F85E000844A4F860000021304680
:10B3A000F5F710FC00213846F5F70CFC01231A468E
:10B3B00005218FE619461046FAF72AFE2860B5F9EE
:10B3C000020040F68151484380136880B5F90010AF
:10B3D00040F68152514389134218A2F681525242DB
:10B3E00029805210A4F85E201044A4F8620008449A
:10B3F000A4F86000002100E091E03046F5F7E2FBA0
:10B4000000213846F5F7DEFB01231A460721DCE66A
:10B410005942404209B200B2FAF7FAFD2860B5F984
:10B42000020040F68151484380136880B5F900104E
:10B4300040F68152514389134218A2F6815252427A
:10B4400052102980A4F85E201044A4F8600008443B
:10B45000A4F8620000213046F5F7B4FB002138461D
:10B46000F5F7B0FB01231A460621AEE61146FAF7BE
:10B47000CFFD2860B5F9020040F6815148438013A2
:10B480006880B5F9001040F6815251438913421883
:10B49000A2F68152524252102980A4F86020104432
:10B4A000A4F85E000844A4F8620000213046F5F7D5
:10B4B00089FB00213846F5F785FB01231A46052153
:10B4C000E3E6504201B2584200B2FAF7A1FD28600B
:10B4D000B5F9020040F68151484381136980B5F9FE
:10B4E000000040F68152504380130A18A2F68152A0
:10B4F0005242288052101144A4F86020A4F862102F
:10B500000844A4F85E0000213046F5F75BFB0021FB
:10B510003846F5F757FB01231A460721B5E6002800
:10B5200001DAA4F86490614502DDA4F866C003E086
:10B53000002901DAA4F86690674502DDA4F868C026
:10B5400003E0002F01DAA4F86890297E1848012949
:10B550001AD00680438082801549028808310A800B
:10B5600042884A80808888801148896A08308847E4
:10B5700098F83E00444678B1F7F722F814F83E0FE9
:10B58000401E2070BDE8F09F34F8641F0180618880
:10B590004180A1888180DFE706480088A0F5D0417E
:10B5A0006839EFD0BDE8F05FF7F74CBE840B0020A0
:10B5B0002C000020182C01402DE9F0419E4C9F48A2
:10B5C000B4F862100288511A89B20F2974D3008826
:10B5D000A4F862009A480088DFF86882C0074FF03C
:10B5E00000054FF0010745D0954AD4E90C102432EC
:10B5F0001388B1EB530F02D21288511A08444FF44A
:10B60000F371884200D208468F49B1FBF0F0616CBB
:10B61000C1F35101084406466064F4F70CFF0022B0
:10B620008A4BF4F774FE4FF04042894BF4F76FFEFB
:10B630000E22F4F7DBFEF4F735FFA4F8AC0094F823
:10B640006D008049401CC0B284F86D0091F84A102A
:10B65000082836D3784808380278914201D0017022
:10B6600085807C4A92F800C07B4ABCF1000F04D070
:10B67000858022E0656425657DE0D8F89830A3F5E3
:10B68000FA639E4212DDE36D03F1020C664505DDAF
:10B69000B0F904300A2B0DDA5B1C06E09E4205DA95
:10B6A000B0F90430002B08DD5B1E8380B0F9040084
:10B6B0000A2802DB177001E0BAE01570E66584F82D
:10B6C0006D5066480278C2F381034FF4A542012B06
:10B6D00017D0022B18D045F208232381A4F8A82004
:10B6E000B0F924009BB258438013A4F8A4005C482E
:10B6F00080785FEA407C5948B0F90E0007D551B90F
:10B7000005E045F6C053E8E744F25063E5E706FB81
:10B7100000F1B1FBF3F17043B0FBF3F35149D4F8FE
:10B7200050C0C3F3D1030988CCEBCC0C4FEACC2C2E
:10B7300003EB9C33B0032365B0FBF1F14A4BC9081E
:10B74000B3F846C0CCEBCC0C4FEACC2C01EB9C31CF
:10B75000A3F84610F117890341EA96410023F4F754
:10B76000E1FCB4F8AA10C1EBC101C902C00800EBAA
:10B770009130A4F8AA00616C206F0844206794F807
:10B780007420521CD2B284F87420082A05D3C00851
:10B79000A4F8760084F874502567344AD388580694
:10B7A00005D498F80F00022809D0A4F88A5022483E
:10B7B00094F83F20B8300C2A24D2C57423E094F8C2
:10B7C000380094F88E60B0420CD084F88E0094F863
:10B7D0003D0000F00106C0F34000864202D1A4F80B
:10B7E0008A5005E0B4F88A0040F6B836B04205D277
:10B7F000B4F88A00401CA4F88A00D8E743F080001F
:10B80000D080D4E7C7741A4B41F2482641F2504C1D
:10B8100093F83C400B4B0C2AB3F886300AD3B14264
:10B8200008DB012C06D0614502DD002B00D18774B6
:10B83000BDE8F0818574FBE7500100207807002007
:10B8400000040040C00200204564BD0100209C406F
:10B85000133B33401604002017040020EC040020A2
:10B86000BF07002046010020780A0020480C002075
:10B870005805002070B5394C394821880288511A82
:10B8800089B23E294DD30088364E20803649307823
:10B8900006F1140518B3488B80002880E968284613
:10B8A0008847B5F904003149FCF7C2FB304A608093
:10B8B0004FF48045D3884FF000015E0737D4B0F5D0
:10B8C000F05F2FDDE079401CC0B2E0710A283ED362
:10B8D00043F4004040F00400D080A16036E0888B43
:10B8E000204A8000121D1080888B80005080888B39
:10B8F000800000B290804A8B92002A804A8B92008E
:10B900006A80498B8900A98018497C31FCF790FB3B
:10B91000A080B5F904001549FCF78AFB608001207E
:10B92000307070BD23F40040A560D0800EE043F479
:10B93000004343F00403A160D380B0F5C85F06DC88
:10B9400023F4004020F00400D080A560E171D4E928
:10B950000201884200DB0846206170BD440E0020D1
:10B9600078070020C4060020C002002078C5000827
:10B97000480C002005494FF48040C8608860086189
:10B980000348C18821F48271C1807047440E0020B1
:10B99000480C00202DE9F041404C414E414F2078A9
:10B9A00041F23331C2074FF000050CD0A28962B3D7
:10B9B00094F90700002800DA4042C0B2032829D2D7
:10B9C00040F233302AE0A570E573374AE571A5816E
:10B9D00092F83830237220F00800A18040F0020075
:10B9E0002070BD867560B560F560116D490005D0A9
:10B9F00041F68461A18140F010002070C0B240F097
:10BA0000010020706574BDE8F081658120F01000B0
:10BA1000207024E0042803D240F2666060811EE0BA
:10BA2000052802D240F69910F8E740F6CC420628E5
:10BA300001D3072801D2628111E0082802D24FF415
:10BA40008050EBE7092809D30A2807D341F6CC41F7
:10BA50000B2803D30C2801D342F26661618197F869
:10BA6000A10098B9B088102301B2B4F90A003622B7
:10BA7000FBF730FB7060F168401AB1680844B060B1
:10BA8000B6F900104843C013F060B886B88E10B104
:10BA90000120A070B7E7A570B5E70000580E0020A0
:10BAA000E8060020C0020020500100202DE9F041EE
:10BAB0004C4C2678F0077CD04B48217A4B4D90F8BF
:10BAC0003800814267D04A4A2346DFF828C1575CD4
:10BAD00093F90E2093F90730874203D01CF80170C8
:10BAE000874213D146F002065B1C26705BB2E371FD
:10BAF0001CF80110814201D15B1CE37194F907101D
:10BB0000062901DD0621E171521C1CE03A4F17F8AD
:10BB100001C03A4F844503D017F801C0844513D1C2
:10BB200026F002065B1E26705BB2E371795C8142EF
:10BB300001D15B1EE37194F907306FF005018B4270
:10BB400000DAE171521EA273207294F907108A1C68
:10BB5000042A02D941F68462A281234A012912787B
:10BB60000ADD224B56079B6802D543F0080301E02B
:10BB700023F00803AB606070B1F1FF3F09DA5107B1
:10BB8000A96802D521F0080101E041F00801A9608F
:10BB90006070F7F7DFFEA089002630B1401E000478
:10BBA000000CA08101D1E671A673E87B04280ED0B9
:10BBB00000E00CE0B5F93410512341220020FBF7DE
:10BBC00089FAA886002802D1E07B10B1A670BDE8F2
:10BBD000F0810B4806700B480670207820F00100B9
:10BBE0002070F4E7580E002050010020C002002011
:10BBF00070C6000876C6000882C6000888C600081D
:10BC00008C0700206F070020F0B415460D4A0E4641
:10BC10004FF0FF31B0EBA20F12DA002810DB0A4917
:10BC2000096851F82000406844682CB12946304624
:10BC3000A446F0BC1A4660476FF00500F0BC7047A0
:10BC40000846FBE704000000AC0800200020E412D6
:10BC5000FB0911058B024601A300510029001400C5
:10BC60000A00050003000100173E573CBB3A3E396D
:10BC7000DD37943661354134333335324431613008
:10BC80008A2FBD2EFB2D412DCC1C58585868991970
:10BC9000585858683313005695130054B613005281
:10BCA0005A140050FD14004EA115004C4516004AD0
:10BCB000761600486C17004672180044BA19004204
:10BCC000741B0040911D003EB420003C9F22003AAE
:10BCD000E1220038532300368B24003481250032C2
:10BCE0002B2700302028002E5829002CB02A002AAB
:10BCF0009B2C0028D22D00267C2F002426310022E8
:10BD000002330020FD34001E5C37001CCC3C001ABE
:10BD1000873E0018BE3F001600400014004000128D
:10BD2000004000100040000E0040000C0040000ADF
:10BD300000400008004000060040000400400002EF
:10BD40000040000001020304050005000102030495
:10BD50000104000305020000F001000036010000AC
:10BD6000F8000000BA0000007C0000007C00000029
:10BD70007C000000C91C9C19991CCC199C1CC91979
:10BD80000000290052007B00A400CC00F5001E0139
:10BD9000470170019901C201EA0113023C026502E8
:10BDA0008E02B602DF020803300359038203AA039E
:10BDB000D303FB0324044C0475049D04C504EE0462
:10BDC00016053E0567058F05B705DF0507062F0633
:10BDD00057067F06A706CE06F6061E0746076D071E
:10BDE0009507BC07E4070B08320859088108A80822
:10BDF000CF08F6081D0944096A099109B809DE0946
:10BE0000050A2B0A520A780A9E0AC40AEA0A100B8B
:10BE1000360B5C0B820BA80BCD0BF30B180C3E0CF6
:10BE2000630C880CAD0CD20CF70C1C0D410D650D8C
:10BE30008A0DAF0DD30DF70D1C0E400E640E880E4B
:10BE4000AC0ECF0EF30E170F3A0F5E0F810FA40F3B
:10BE5000C70FEA0F0D103010531075109810BA105C
:10BE6000DD10FF102111431165118711A911CA11AD
:10BE7000EC110D122E12501271129212B312D41232
:10BE8000F41215133613561376139613B713D713EC
:10BE9000F61316143614561475149414B414D314DB
:10BEA000F214111530154E156D158C15AA15C815FF
:10BEB000E7150516231641165F167C169A16B71657
:10BEC000D516F2160F172C17491766178317A017E8
:10BED000BC17D917F51711182E184A1866188118AB
:10BEE0009D18B918D418F0180B19261942195D19A4
:10BEF00078199219AD19C819E219FD19171A311AD2
:10BF00004C1A661A801A991AB31ACD1AE61A001B2F
:10BF1000191B331B4C1B651B7E1B971BAF1BC81BC0
:10BF2000E11BF91B121C2A1C421C5A1C721C8A1C85
:10BF3000A21CBA1CD21CE91C011D181D301D471D76
:10BF40005E1D751D8C1DA31DBA1DD01DE71DFD1D99
:10BF5000141E2A1E401E571E6D1E831E981EAE1EE6
:10BF6000C41EDA1EEF1E051F1A1F2F1F451F5A1F62
:10BF70006F1F841F991FAE1FC21FD71FEC1F002009
:10BF800000006400C9002D019201F7015B02C002AC
:10BF900024038903ED035204B6041A057F05E30563
:10BFA0004706AB060F077307D7073B089F08020930
:10BFB0006609C9092D0A900AF30A560BB90B1C0C25
:10BFC0007F0CE20C440DA60D090E6B0ECD0E2F0F4B
:10BFD000900FF20F5310B41015117611D7113812BB
:10BFE0009812F8125813B81318147714D61435157C
:10BFF0009415F3155116B0160E176B17C91726189E
:10C000008318E0183D199919F519511AAD1A081B32
:10C01000631BBE1B181C731CCD1C261D801DD91D47
:10C02000321E8A1EE31E3B1F921FEA1F41209820EA
:10C03000EE2044219A21EF2145229922EE2242232B
:10C040009623E9233C248F24E22434258525D72513
:10C0500028267826C82618276827B72706285428B0
:10C06000A228EF283D298929D629222A6D2AB82A13
:10C07000032B4D2B972BE12B2A2C722CBB2C022D42
:10C080004A2D912DD72D1D2E632EA82EEC2E302F4C
:10C09000742FB82FFA2F3D307F30C030013141313D
:10C0A0008131C13100323F327D32BA32F73234331E
:10C0B0007033AC33E73322345C349534CE340735F7
:10C0C0003F357735AE35E4351A3650368536B936D4
:10C0D000ED36203753378637B737E93719384938BF
:10C0E0007938A838D738053932395F398B39B739BB
:10C0F000E2390D3A373A603A893AB23ADA3A013BD4
:10C10000283B4E3B733B983BBD3BE03B043C263C0D
:10C11000483C6A3C8B3CAB3CCB3CEA3C093D273D70
:10C12000443D613D7D3D993DB43DCE3DE83D013E00
:10C130001A3E323E493E603E763E8C3EA13EB53EC2
:10C14000C93EDC3EEF3E013F123F233F333F433FBA
:10C15000513F603F6E3F7B3F873F933F9E3FA93FEC
:10C16000B33FBC3FC53FCD3FD53FDC3FE23FE83F5B
:10C17000ED3FF13FF53FF93FFB3FFD3FFF3FFF3F05
:10C18000FF3F0000E0203420002020E0202020237A
:10C190003720262021000080020004000800100043
:10C1A000000200040008040000020004000800105F
:10C1B00000200040008004000000008000000040DB
:10C1C0000000002000000010000000080000000433
:10C1D000000000020000000100008000000040009C
:10C1E0000000200000001000000008000000040013
:10C1F0000000020000000100008000000008014073
:10C20000000C0140000C0140000C0140000C0140FA
:10C21000000C0140000C0140000C014000100140E6
:10C2200000100140001001400010014000100140CA
:10C2300000100140001001400010014000140140B6
:10C2400004080140040C0140040C0140040C0140AE
:10C25000040C0140040C0140040C0140040C01409A
:10C26000041001400410014004100140041001407A
:10C27000041001400410014004100140041001406A
:10C280000414014008080140080C0140080C01405A
:10C29000080C0140080C0140080C0140080C01404A
:10C2A000080C01400810014008100140081001402E
:10C2B000081001400810014008100140081001401A
:10C2C00008100140081401400C0801400C0C01400A
:10C2D0000C0C01400C0C01400C0C01400C0C0140FA
:10C2E0000C0C01400C0C01400C1001400C100140E2
:10C2F0000C1001400C1001400C1001400C100140CA
:10C300000C1001400C1001400C14014010080140B9
:10C31000100C0140100C0140100C0140100C0140A9
:10C32000100C0140100C0140100C01401010014095
:10C330001010014010100140101001401010014079
:10C340001010014010100140101001401014014065
:10C3500000000000000000000000000000000000DD
:10C360000000000014080140140C0140140C0140AE
:10C37000140C0140140C0140140C0140140C014039
:10C38000140C01401410014014100140141001401D
:10C390001410014014100140141001401410014009
:10C3A00014100140141401400000000000000000BF
:10C3B000000000000000000000000000FFFFFF0F71
:10C3C0000FFFFFFFFFF0FFFFFF0FFFFFFFFFF0FF7B
:10C3D0000FFFFFFFFFF0FFFFFF0FFFFFFFF0FFFF6B
:10C3E0000FFFFFFFFFF0FFFFFF0FFFFFFFFFF0FF5B
:10C3F000FFFF0FFFFFFFFFF0FFFFFF0FFFF0FFFF4B
:10C400000000004040000000000400000040000068
:10C410000000040040000000000400000040000094
:10C420000004000040000000000400000040000084
:10C430000000040000004000000000040000004074
:10C4400000040000000000808000000000080000E0
:10C4500000800000000008008000000000080000CC
:10C4600000800000000800008000000000080000BC
:10C4700000800000000008000000800000000008AC
:10C4800000000080000800000000002020000000E4
:10C490000002000000200000000002002000000058
:10C4A0000002000000200000000200002000000048
:10C4B0000002000000200000000002000000200038
:10C4C00000000002000000200002000000000060E8
:10C4D0006000000000060000006000000000060090
:10C4E0006000000000060000006000000006000080
:10C4F0006000000000060000006000000000060070
:10C50000000060000000000600000060000600005F
:10C51000008002000400080010000002000400086F
:10C520000400000200040008001000200040008009
:10C5300004000000FF7FFFFFFDFFFFFFFBFFFFFF89
:10C54000F7FFFFFFEFFFFFFFFFFDFFFFFFFBFFFF19
:10C55000FFF7FFFFFBFFFFFFFFFDFFFFFFFBFFFFFD
:10C56000FFF7FFFFFFEFFFFFFFDFFFFFFFBFFFFF53
:10C57000FF7FFFFFFBFFFFFF401FFC02001E5A036F
:10C58000C01CC403801B3C04401AC6040019630588
:10C59000C01717068016E4064015CD070014D7080B
:10C5A000C012050A80115B0B4010DD0C000F900ECD
:10C5B000C00D7510800C9012400BE014000A651736
:10C5C000C0081C1A8007FD1C400600200005182327
:10C5D000C003372680024E2940014C2C0000242F36
:10C5E000C0FEC73180FD2E3400FB2D3880F81C3B87
:10C5F00000F6003C8025151A40249A1B00231E1DBE
:10C60000C021B81E80205D20401F0C22001EC223C6
:10C61000C01C7E25801B3327401AFB280019B72A2F
:10C62000C0176D2C8016192E4015B92F00144731F4
:10C63000C012C9328011353440108B35000FCA3614
:10C64000C00DF037800CFE38400BF439000AD23AA6
:10C65000C008983B8007473C4006E13C0005673D29
:10C66000C003DA3D80023E3E4001923E0000143F8E
:10C670000102030405000203040500010304050090
:10C68000010205000102030404050001020355052F
:10C690000010AA1A55250030AA3A0000AA0A55151A
:10C6A0000020AA2A5535FF3FAA0A55150020AA2ABC
:10C6B0005535FF3F6465765F63616E3100000000B1
:10C6C0000D950008BD960008399600086994000889
:10C6D0003194000800000000B4C60008C0C600087D
:10C6E00004C7000800000020CC0800000007000874
:10C6F00030C80008CC0800204415000064900008F1
:10C70000D8C6000801581369461B087D042113553B
:10C71000152A4006190801A7130B631B0831041AD8
:10C720002B0401288201170206040501031480204E
:10C73000FF8BAA0A0201A415AA0A55150008592060
:10C74000AA2A5535FF3F07350301050406020312E7
:10C750007C1573FFFF04FF808001012D025F6402DE
:10C76000130A13659752081201100C050406020300
:10C77000010103070505280B010203040206070354
:10C7800003040C3D0706040509191F191904310596
:10C7900006060B14AA1A02312E40FD396926021131
:10C7A000042F405F02041E405B2613E8058A202EFA
:10C7B000CD551555154039020187031ED0071AFFC4
:10C7C00001013B0261AA0C10080108A834993F330B
:10C7D00013959F391CA910091EF011220312100A8B
:10C7E00017401C12600A16901B011AA2646B7997FD
:10C7F00094012199D0019A5A14021AC802CBD00789
:10C80000023A19164902892612C8DA01DA1AFF011A
:10C81000C1227D130D0212103AFA0812081CF4010D
:10C82000010812062BE8031022021AC715011B008B
:020000040800F2
:10FC00004A46545A594D46312D4E3330202020203B
:10FC1000050406020301AA0AAA0AAA0AAA0AAA0A4B
:10FC2000AA0ADE3F00100000FF0131000301664612
:10FC300000400040513800400040004000400101B9
:10FC4000004000407A3B082708270827FF0033338D
:10FC50000201401F00016626B81E6626FFFFFFFF57
:10FC6000FFFF01010100010000000300000202008B
:04FC70000000AA5591
:04000005080000ED02
:00000001FF
